:100000000C941E090C9444090C9444090C94440962
:100010000C9444090C9444090C9444090C9444092C
:100020000C9444090C9444090C9481170C942518E1
:100030000C9444090C9444090C9451090C944409FF
:100040000C9444090C9444090C9444090C944409FC
:100050000C94A2160C9444090C9444090C94440981
:100060000C9444090C9444090C9444090C944409DC
:100070000C9444090C9444090C9444090C944409CC
:100080000C9444090C9444090C9444090C944409BC
:100090000C9444090C9444090C9444090C944409AC
:1000A0000C9444090C9444090C9444090C94800960
:1000B0000C9444090C9444090C9444090C94124B7C
:1000C0000C9444090C9444090C9444090C9444097C
:1000D0000C9444090C9444090C9444090C9444096C
:1000E0000C9444090C9444090C9444090C9444095C
:1000F0000C9444090C9444090C9444090C9444094C
:100100000C9444090C9444090C9444090C9444093B
:100110000C9444090C9444090C9444090C9444092B
:100120000C9444090C9444090C9444090C9444091B
:100130000C9444090C9444090C9444090C9444090B
:100140000C9444090C9444090C9444090C945A24CA
:100150000C9444090C9444090C9444090C944409EB
:100160000C9444090C9444090C9444090C944409DB
:100170000C9444090C9444090C9444090C944409CB
:100180000C9444090C9444090C9444090C944409BB
:100190000C9444090C9444090C9444090C944409AB
:1001A0000C9444090C9444090C9444090C9444099B
:1001B0000C9444090C9444090C9444090C9444098B
:1001C0000C9444090C9444090C9494090C9444092B
:1001D0000C9444090C9444090C9444090C940216A0
:1001E0000C94CD150C9444090C9444090C944409C6
:1001F0000C944409BE211F1AD91F9720DE1F1F1A15
:100200003B231F1A8D1D4023B9219B1E1F1AA321BA
:10021000C71F1F1A1F1A1C20A91DDA21B4219E21F5
:10022000F22076224D542D583120584D454741201B
:1002300044656D6F2050726F6772616D0046697220
:100240006D776172652052657620313130393139F0
:10025000006D617474616972746563682E636F6D9B
:10026000004D61696E204D656E7500525443204308
:100270006C6F636B0A54656D70657261747572653D
:100280002053656E736F720A417564696F20416D0A
:10029000706C69666965720A534420436172640A2E
:1002A00053657269616C205352414D0A4C45447349
:1002B0000A427574746F6E730A52656C61792044DA
:1002C00072697665720A536C6565702044656D6F5E
:1002D0000A4C69766567726170682044656D6F0AC3
:1002E0004144562044656D6F0A314D4220535241BE
:1002F0004D20546573740A437265646974730052C7
:10030000656C617920310A52656C617920320A523C
:10031000656C617920330A52656C617920340A5228
:10032000656C617920350A52656C617920360A5214
:10033000656C617920370A52656C61792038004F0D
:1003400066660A4F6E0043757272656E742054695A
:100350006D653A00546869732064656D6F20697338
:1003600020616C7761797320656E61626C65640AE7
:100370005573652074686520627574746F6E7320A0
:10038000746F206E61766967617465207468657347
:1003900065206D656E7573004E6F7720696E2073F2
:1003A0006C656570206D6F64650A525443207761F7
:1003B0006B696E67206576657279207365636F6E11
:1003C0006420746F207570646174652074696D6554
:1003D0000A50726573732061206D6964646C6520D6
:1003E000627574746F6E20746F2065786974004351
:1003F000757272656E742054656D70657261747586
:1004000072653A0053746172742044656D6F0A53CB
:10041000746F702044656D6F005072657373206156
:100420006E79206B657920746F20626567696E2034
:1004300073656E64696E67204C697665677261707A
:100440006820646174612E0A50726573732061675D
:1004500061696E20746F2073746F7020616E642008
:1004600072657475726E20746F206D61696E206D97
:10047000656E752E00312920446973636F6E6E6559
:100480006374207465726D696E616C0A3229205341
:1004900074617274204144562C2073656C656374DA
:1004A00020434F4D20706F72742C204F4B0A33291C
:1004B00020436C69636B20677265656E20537461BD
:1004C000727420627574746F6E0A342920507265DC
:1004D000737320627574746F6E2032206F722033D4
:1004E00020746F20626567696E2073656E64696E43
:1004F0006720646174610A342920436C69636B204E
:100500002753686F7720436F6E66696775726174F1
:10051000696F6E20506172616D6574657273270A30
:1005200035292056696577206461746120627920DD
:1005300073656C656374696E6720746162730A36F3
:100540002920436C69636B207265642073746F703B
:1005500020627574746F6E2C20636C6F736520411C
:1005600044560A37292052652D636F6E6E65637499
:10057000207465726D696E616C0A3829205072654D
:100580007373203C656E7465723E20746F207374C3
:100590006F702073656E64696E6720616E6420728F
:1005A000657475726E20746F206D61696E206D6563
:1005B0006E75005352414D2054657374205375631A
:1005C0006365737366756C210044656D6F206861A7
:1005D00073206E6F74206265656E20777269747423
:1005E000656E0A436865636B20776562736974653D
:1005F00020736F6F6E21004A757374696E204D61B0
:1006000074746169720A4465616E2043616D65723C
:1006100061202D20555342206C6962726172792CE1
:10062000205044492070726F6772616D6D65720A67
:100630004368614E202D2046617446532C2053445C
:100640002043617264206472697665720A50657431
:100650006572204B77616E202D2053657269616C45
:100660002052414D0A41746D656C20436F72706F6A
:10067000726174696F6E202D2053616D706C6520FE
:1006800044726976657273005352414D20646174FF
:100690006120696E7465677269747920746573741A
:1006A000206661696C757265206174206164647292
:1006B00065737320307825580A005352414D2064E9
:1006C00061746120696E74656772697479207465FC
:1006D00073742073756363657373210A0053524109
:1006E0004D20616464726573732062757320746554
:1006F0007374206661696C75726520617420616431
:10070000647265737320307825580A005352414D46
:1007100020616464726573732062757320746573FD
:10072000742073756363657373210A005352414DDE
:10073000206461746120627573207465737420662F
:1007400061696C757265206174206164647265739F
:100750007320307825580A005352414D206461744B
:1007600061206275732074657374207375636365AB
:100770007373210A002532642E253032640A005436
:10078000656D7065726174757265202843290A0071
:10079000404D542D5831204C697665677261706800
:1007A0002054656D70657261747572652044656D65
:1007B0006F0A002533642E25303264432020202028
:1007C000202533642E25303264460A002020202064
:1007D00020202531642E25303464560A0025752FDB
:1007E00025752F257520253032753A253032753A1A
:1007F000253032750A0068202D2068656C700A006B
:1008000078202D20657869740A0074205B3C796536
:1008100061723E203C6D6F6E3E203C6D6461793E9E
:10082000203C686F75723E203C6D696E3E203C73C3
:1008300065633E5D202D206C6973742F6368616E63
:100840006765205254432074696D650A00666A200A
:100850003C6472697665233E202D204368616E6793
:10086000652063757272656E742064726976650ABC
:10087000006667203C706174683E202D20436861EB
:100880006E67652063757272656E74206469726547
:1008900063746F72790A006678203C7372635F6ECE
:1008A000616D653E203C6473745F6E616D653E20D2
:1008B0002D20436F70792066696C650A006674208C
:1008C0003C796561723E203C6D6F6E74683E203CE1
:1008D0006461793E203C686F75723E203C6D696EA4
:1008E0003E203C7365633E203C6E616D653E0A00B0
:1008F0006661203C617472723E203C6D61736B3E98
:10090000203C6E616D653E202D204368616E6765F9
:100910002066696C652F6469722061747472696203
:100920007574650A00666B203C6E616D653E202D16
:100930002043726561746520612064697265637427
:100940006F72790A006675203C6E616D653E202DE0
:1009500020556E6C696E6B20612066696C65206F36
:1009600072206469720A00666E203C6F6C645F6E70
:10097000616D653E203C6E65775F6E616D653E2002
:100980002D204368616E67652066696C652F646918
:1009900072206E616D650A006676202D2054727596
:1009A0006E636174652066696C650A006677203C39
:1009B0006C656E3E203C76616C3E202D207772691E
:1009C00074652066696C650A006664203C6C656E1F
:1009D0003E202D207265616420616E642064756D17
:1009E000702066696C652066726F6D206375727227
:1009F000656E742066700A006672203C6C656E3EFF
:100A0000202D20726561642066696C650A00666548
:100A1000203C706F736974696F6E3E202D205365A2
:100A2000656B2066696C6520706F696E7465720A0B
:100A3000006663202D20436C6F736520612066691A
:100A40006C650A00666F203C6D6F64653E203C6EED
:100A5000616D653E202D204F70656E2061206669B6
:100A60006C65202869653A20666F20312046494C24
:100A7000452E545854290A00666C205B3C70617402
:100A8000683E5D202D204469726563746F72792021
:100A90006C697374696E670A006673205B3C7061F1
:100AA00074683E5D202D2053686F77206C6F6769F6
:100AB00063616C2064726976652073746174757308
:100AC0000A006669203C6C6F6720647276233E20C2
:100AD0002D20496E697469616C697A65206C6F6755
:100AE0006963616C2064726976650A006266203C05
:100AF0006E3E202D2046696C6C20776F726B696E9C
:100B000067206275666665720A006277203C7068CD
:100B1000795F647276233E203C736563746F723E26
:100B2000205B3C6E3E5D202D20577269746520521B
:100B30002F572062756666657220696E746F206437
:100B400069736B0A006272203C7068795F64727628
:100B5000233E203C736563746F723E205B3C6E3EA7
:100B60005D202D2052656164206469736B20696E7D
:100B7000746F20522F57206275666665720A006294
:100B800065203C616464723E205B3C646174613E3C
:100B90005D202E2E2E202D204564697420522F5763
:100BA000206275666665720A006264203C61646456
:100BB000723E202D2044756D7020522F5720627593
:100BC000666665720A006473203C7068795F6472BF
:100BD00076233E202D2053686F77206469736B2045
:100BE0007374617475730A006469203C7068795F7E
:100BF000647276233E202D20496E697469616C69A8
:100C00007A65206469736B0A006464203C706879BB
:100C10005F647276233E205B3C736563746F723E43
:100C20005D202D2044756D7020736563746F720AAA
:100C30000025752F25752F257520253032753A250D
:100C40003032753A253032750A000A256C752062FB
:100C50007974657320636F706965642E0A000A43B6
:100C60006F7079696E672E2E2E000A43726561746B
:100C7000696E672022257322004F70656E696E676A
:100C8000202225732200256C7520627974657320FB
:100C90007772697474656E207769746820256C7545
:100CA0002062797465732F7365632E0A00256C7555
:100CB0002062797465732072656164207769746855
:100CC00020256C752062797465732F7365632E0A15
:100CD0000066707472203D20256C75283078256C74
:100CE00058290A002C202531306C754B206279740C
:100CF000657320667265650A002534752046696C47
:100D0000652873292C2531306C75206279746573E0
:100D100020746F74616C0A253475204469722873DD
:100D20002900256325632563256325632025752F09
:100D3000253032752F2530327520253032753A2511
:100D40003032752025396C7520202573000D2575EE
:100D50002066696C65732C20256C7520627974653A
:100D6000732E0A257520666F6C646572732E0A25D2
:100D70006C75204B4220746F74616C206469736BD6
:100D80002073706163652E0A256C75204B422061CB
:100D90007661696C61626C652E0A0046415420746C
:100DA000797065203D2025750A42797465732F435B
:100DB0006C7573746572203D20256C750A4E756DD7
:100DC000626572206F662046415473203D20257570
:100DD0000A526F6F742044495220656E74726965BF
:100DE00073203D2025750A536563746F72732F4617
:100DF0004154203D20256C750A4E756D6265722048
:100E00006F6620636C757374657273203D20256C6A
:100E1000750A46415420737461727420286C6261B3
:100E200029203D20256C750A444952207374617253
:100E30007420286C62612C636C7573746F72292046
:100E40003D20256C750A446174612073746172746D
:100E500020286C626129203D20256C750A0A2E2EFF
:100E60002E0072633D25750A0072633D25750A00E8
:100E70003F3F3F0A002530345820253032582D009E
:100E8000532F4E3A2025730A004D6F64656C3A204B
:100E900025730A005344205374617475733A0A0031
:100EA0004F43523A0A004349443A0A004353443AF2
:100EB0000A004361726420747970653A2025750ACE
:100EC00000457261736520626C6F636B2073697A91
:100ED000653A20256C7520736563746F72730A0020
:100EE000536563746F722073697A653A2025750AB9
:100EF0000044726976652073697A653A20256C75BD
:100F000020736563746F72730A0072633D25640A0F
:100F100000536563746F723A256C750A0072633D05
:100F200025640A0027682720666F722068656C7048
:100F30002C2027782720666F7220657869740A0054
:100F4000546F20626567696E3A206469303C656E53
:100F50007465723E206669303C656E7465723E0A47
:100F60000046617446732052302E30376420746519
:100F70007374206D6F6E69746F7220666F72205388
:100F8000442F4D4D430A002025303258002530387B
:100F90006C58200072633D25752046525F25530A28
:100FA000004F4B004449534B5F45525200494E5449
:100FB0005F455252004E4F545F5245414459004ED6
:100FC0004F5F46494C45004E4F5F504154480049E1
:100FD0004E56414C49445F4E414D450044454E49B3
:100FE000454400455849535400494E56414C4944E4
:100FF0005F4F424A4543540057524954455F50524F
:101000004F54454354454400494E56414C49445F72
:101010004452495645004E4F545F454E41424C455F
:1010200044004E4F5F46494C455F53595354454D1C
:10103000004D4B46535F41424F5254454400544982
:101040004D454F55540000507265737320616E79A1
:10105000206B6579004261636B00204F4B200020BC
:1010600043414E43454C20004E657720686578200B
:1010700076616C75653A00417564696F2044656DF1
:101080006F005741562046696C650A566F6C756D46
:10109000650A506C61796261636B0A457869740016
:1010A0005741562046696C6520496E666F726D61C6
:1010B00074696F6E0046696C656E616D650A536197
:1010C0006D706C65726174650A5265736F6C7574CE
:1010D000696F6E0A4368616E6E656C730053656C70
:1010E000656374205741562066696C6500457272CD
:1010F0006F722100436F756C64206E6F74206D6F8A
:10110000756E7420534420636172640046617446B6
:1011100053204572726F7200496E76616C6964206B
:101120005741562046696C6500506C6179696E675D
:101130000053746F70706564006461746100666D63
:101140007420005741564500524946460025632009
:10115000253134730044202E2E002E2E005072654F
:10116000737320616C6D6F737420616E79206B6591
:101170007920746F20636F6E74696E75650A0D0A4D
:101180000D0052656164696E672074686520646152
:101190007461206261636B0A0D0057726974696E35
:1011A0006720646174613A0A0D0052656164696E7A
:1011B00067206261636B2074686520737461747565
:1011C000732076616C75653D253033640A0D0053DC
:1011D000657474696E6720746865207374617475D2
:1011E0007320746F2036340A0D0053504920524149
:1011F0004D2044656D6F20537461727465640A00FC
:10120000476F7420253033640A0D0053656E64699E
:101210006E6720253033640A0D00454647656667D2
:1012200000202B2D2E3031323334353637383968A3
:10123000006364696E6F70737578580011241FBE67
:10124000CFEFDFE3DEBFCDBF00E00CBF18BE19BE9D
:101250001ABE1BBE10E2A0E0B0E2EEEAFBEB00E03B
:101260000BBF02C007900D92A63BB107D9F71BBE7A
:1012700014E3A6EBB0E201C01D92A43FB107E1F771
:101280000E9452110C94D55D0C94000084EC99E0FE
:1012900020E233E0F9013197F1F70197D9F782E0C5
:1012A00008951F920F920FB60F9208B60F9209B6CB
:1012B0000F92112418BE19BE8F939F93AF93BF93C3
:1012C0008091C9209091CA20A091CB20B091CC20D0
:1012D0000196A11DB11D8093C9209093CA20A093AF
:1012E000CB20B093CC20BF91AF919F918F910F9065
:1012F00009BE0F9008BE0F900FBE0F901F9018955B
:101300001F920F920FB60F9208B60F92112418BEBB
:101310008F9381E08093D0208F910F9008BE0F9023
:101320000FBE0F901F9018951F920F920FB60F923D
:1013300008B60F9209B60F920BB60F92112418BE81
:1013400019BE1BBE2F933F934F935F936F937F9371
:101350008F939F93AF93BF93EF93FF938091CE2092
:10136000813011F482E001C084E08093CE2080E4DB
:101370009BE060E00E94CA11FF91EF91BF91AF9195
:101380009F918F917F916F915F914F913F912F919D
:101390000F900BBE0F9009BE0F9008BE0F900FBEAE
:1013A0000F901F90189581E061E00E9401468AE24B
:1013B00060E50E943C4582E06CE10E94014684E2C7
:1013C00092E00E94E44583E06EE10E9401468DE3D5
:1013D00092E00E94E44584E060E20E94014681E5DB
:1013E00092E00E94E44585E061E00E9401468AE2C5
:1013F00060E50E943C45089582E591E20E9408154F
:1014000008951F93182F82E591E2612F0E94DF1447
:101410008823C9F31F9108954F925F926F927F9234
:101420008F929F92AF92BF92CF92DF92EF92FF92F4
:101430000F931F9380914800817F866080934800BE
:101440000E94931580E096E06FEF40E020E000E01E
:1014500077E0E72E0E94901380E296E06FE040E094
:1014600020E00E94901388248A948092B00098E132
:10147000E0E4F6E0908B81E48093B00050EAC52E62
:1014800056E0D52EF601908B8092B00040EE442EAF
:1014900046E0542EF201908B8092B000E0E2F7E03B
:1014A000908B81E08093B000E0EEF7E0908B30E627
:1014B000A32E36E0B32E8FE0F5018683818320E8EA
:1014C000622E26E0722EF301828380E896E06FE0C0
:1014D00040E020E008E1EE240E949013E0ECF7E009
:1014E00098E0F92EF682F18284E0982E958291821E
:1014F00010E1F601128380EA96E060E140E020E02E
:101500000E949013F50115831183F3011583118354
:10151000F601F582F182928280EA96E064E040E092
:1015200020E00E94901382E0F601828380EA96E038
:1015300062E040E020E00E94901380E4F3018283A7
:1015400080E896E060E440E020E00E94901380E2B2
:10155000F6018583818380E8858381831092CE2084
:1015600083EFF20184838092E0068092200780E47A
:1015700060E048E021E00E94B65280E594E060E33C
:1015800040E050E422E00E94BC5280915000826012
:10159000809350008091510081FFFCCF80E868E08B
:1015A0000E94E5138091500080618093500080E09C
:1015B00061E00E94F5138091510084FFFCCF84E02C
:1015C0000E940D1480E060E042E00E94DA138091F6
:1015D00050008860809350008091510083FFFCCFC1
:1015E00082E00E942A148091010480FDFCCF80E0FB
:1015F00094E060E070E041E050E021E00E9481145E
:1016000081E064E00E949D140E945B1781E061E02C
:101610000E94321482E061E00E943214E0EAF0E0BD
:101620008091A200816082838091A2008260828387
:101630008091A200846082838091A200806882836E
:1016400078941F910F91FF90EF90DF90CF90BF9013
:10165000AF909F908F907F906F905F904F90089584
:101660001F938091880680958F70823061F083305F
:1016700020F4813009F05BC008C0843021F088304C
:1016800009F055C004C01DE003C012E401C011E41C
:101690008091CE208823C1F4E0E4FBE088E08187DC
:1016A00082EA93E086A397A380E49BE061E00E9436
:1016B0000A1280E49BE067E00E94CA111093D120D7
:1016C00081E08093CE202FC08091CE20823059F4CB
:1016D0008091D120181729F5E0E4FBE088E08187AC
:1016E0008CE89CE30AC08091CE208430E1F4E0E4F1
:1016F000FBE088E081878CE19CE086A397A380E4EF
:101700009BE061E00E940A1280E49BE067E00E9497
:10171000CA1183E08093CE2007C08091CE20813013
:1017200011F01092CE2010E0812F1F91089580912A
:10173000CE20882391F7F7CFCF93DF93EC012BC016
:101740008091C520882329F00E94564B88838823E6
:1017500079F580912720882339F00E94300B888307
:101760008D3021F1882321F58091CF20882321F02D
:101770000E9433178823E1F48091CD20882359F00B
:101780008091D020882339F40E944D167894889552
:1017900000000E94691682E591E20E9408158823E4
:1017A00079F282E591E20E941215888380E001C0FF
:1017B00081E0DF91CF9108950F93482F89EC95E058
:1017C0006BE672E024E001E00E9425460F91089547
:1017D0000F9387EF95E06BE672E04CE024E001E0C8
:1017E0000E9425460F9108950F9384E593E06BE6E0
:1017F00072E046E024E001E00E9425460F91089542
:10180000EF92FF920F9381E08093CD201092D02031
:10181000E8E4EE2EF12CF70180818160808380E87E
:1018200096E062E04FE00E94821388E993E06BE665
:1018300072E048E024E001E00E94254680E896E05E
:1018400060E04FE00E948213F70180818E7F8083E9
:101850001092CD200F91FF90EF9008950F938AEE94
:1018600094E48093C7209093C82080EE9BE28093FD
:10187000DE2B9093DF2B60E070E480E090E00E942C
:10188000E8549B01AC012F3F8FEF38078FEF4807DB
:101890008FEF580769F40F920F9288E597E0EDB744
:1018A000FEB7818392830E941B580F900F9013C044
:1018B00000D000D08CE297E0EDB7FEB78183928331
:1018C00023833483458356830E941B588DB79EB76C
:1018D00006968DBF9EBF60E070E480E090E020E05F
:1018E00030EC4FE050E00E9465539B01AC012F3F6C
:1018F0009FEF39079FEF49079FEF590769F40F9250
:101900000F928CE097E0EDB7FEB7818392830E943F
:101910001B580F900F9013C000D000D08DED96E0B3
:10192000EDB7FEB781839283238334834583568347
:101930000E941B588DB79EB706968DBF9EBF60E074
:1019400070E480E090E020E030EC4FE050E00E9456
:101950001D549B01AC012F3F9FEF39079FEF4907B3
:101960009FEF590769F40F920F928AEB96E0EDB75B
:10197000FEB7818392830E941B580F900F9013C073
:1019800000D000D088E896E0EDB7FEB7818392835F
:1019900023833483458356830E941B588DB79EB79B
:1019A00006968DBF9EBFE091DE2BF091DF2B11924A
:1019B000E093DE2BF093DF2B80E090E06BE672E0AB
:1019C0004BE024E001E00E9425460F9108952F92FC
:1019D0003F924F925F926F927F928F929F92AF92BF
:1019E000BF92CF92DF92EF92FF920F931F93DF93FC
:1019F000CF93CDB7DEB7C856D040CDBFDEBF8FEF97
:101A000089839AE59A83E8E0F0E0EB83FC83FF2486
:101A1000F394FD82F2E0FE831F8286E08887CE0188
:101A2000019668E070E00E943F579FEF998BEAE5CE
:101A3000EA8B83E08D8B82E19AE7A0E0B0E08F8BA8
:101A4000988FA98FBA8F86E290E08B8B9C8BF6E003
:101A5000FEAB1DAA8FEF8FABE8AF94E0E92EEBAEA3
:101A600082E390E089AF9AAFEEAEFFAEFE01E85997
:101A7000FF4F96E09083FE01E959FF4F1082FE8AE6
:101A8000FB8E81E1282E312C2C0E3D1E0CE1402EC8
:101A9000512C4C0E5D1EC20160E070E20E94BF5CE2
:101AA000C10166E270E00E943F57FCAEFDAE10E45B
:101AB000612E712C6C0E7D1E8CEE9FEFAFEFBFEF91
:101AC000F30180839183A283B383B4E48B2E912CA2
:101AD0008C0E9D1E8CE890E0A0E0B0E0F4018083C5
:101AE0009183A283B3838E01095C1F4FA1E1AA2ECB
:101AF000B12CA00EB11EC5016CE070E20E94BF5C6B
:101B0000F5E2CF2ED12CC00ED11EC60162E170E2EB
:101B10000E94BF5CC80162E370E00E943F57F2E0A0
:101B2000FE8BFB8EC20167E170E20E94BF5CC101C7
:101B300066E270E00E943F5782E08CAFFDAEF30199
:101B4000108211821282138284EC99E0A0E0B0E04E
:101B5000F40180839183A283B383C5016FE170E2B6
:101B60000E94BF5CC60162E270E20E94BF5CC801D5
:101B700062E370E00E943F57FFEFF9878AE58A87AA
:101B8000E8E0F0E0EB87FC87F2E0FD87EE861F8659
:101B900086E0888BCE01099668E070E00E943F578E
:101BA000C859DF4FCDBFDEBFCF91DF911F910F919D
:101BB000FF90EF90DF90CF90BF90AF909F908F906D
:101BC0007F906F905F904F903F902F9008958F92ED
:101BD0009F92AF92BF92CF92DF92EF92FF920F93BC
:101BE0001F931092C9201092CA201092CB201092FD
:101BF000CC2082E496E18093C7209093C820E0E057
:101C0000F8E088E0818780E09DE786A397A380E0E5
:101C100098E061E00E94041280E098E061E00E9498
:101C2000C4110E94645185E794E06BE672E04AE0DB
:101C300024E001E00E9425460E94E70C0E94331731
:101C400059C00E943317882309F454C0C090C9209A
:101C5000D090CA20E090CB20F090CC200E9432514E
:101C6000AA2797FDA095BA2FBC01CD0124ED30E342
:101C700040E050E00E94095C20E038E040E050E0A5
:101C80000E94715C49015A0184ED90E3A0E0B0E04C
:101C9000880E991EAA1EBB1EC501B401660F771FD0
:101CA000881F991F680D791D8A1D9B1D605E7E42ED
:101CB0008040904025E431E040E050E00E94715CBB
:101CC00089019A01005E1F4F2F4F3F4F81E0A6010F
:101CD000B7010E949D57C501B4012AE030E040E001
:101CE00050E00E94715C89019A0182E0A601B7016F
:101CF0000E949D5782E591E20E940815882309F40D
:101D0000A0CF82E591E20E94121580E098E060E0A9
:101D10000E94C4110E9429511F910F91FF90EF90D2
:101D2000DF90CF90BF90AF909F908F900895AF922B
:101D3000BF92CF92DF92EF92FF920F931F93CF93B8
:101D4000DF9382E496E18093C7209093C8200E949D
:101D5000645189E194E06BE672E049E024E001E03F
:101D60000E9425460F920F9280E997E0ADB7BEB76B
:101D700011968D939C9312970E941B588FE797E0C2
:101D8000EDB7FEB7818392830E941B580F900F908E
:101D90000E94331745E7A42E47E0B42E34E6C32E45
:101DA000D12C61C00E943317882309F45CC00E94C3
:101DB0003251AA2797FDA095BA2FBC01CD0124ED81
:101DC00030E340E050E00E94095C20E038E040E071
:101DD00050E00E94715C79018A0100D000D0CDB73B
:101DE000DEB72196ADB7BEB71196AD92BC921297F1
:101DF00084E391E2A0E0B0E0E80EF91E0A1F1B1F89
:101E0000C801B70123EC30E040E050E00E94715C73
:101E10002A833B8380EA9FE0A0E0B0E0E80EF91E51
:101E20000A1F1B1FC701805A9F4097FF03C0909550
:101E300081959F4F63EC70E00E943C5CDC01AC9D9F
:101E4000C001AD9D900DBC9D900D112463EC70E020
:101E50000E943C5C6C837D830E941B58EDB7FEB7EB
:101E60003696EDBFFEBF82E591E20E9408158823F9
:101E700009F498CF82E591E20E9412150E9429513F
:101E8000DF91CF911F910F91FF90EF90DF90CF9056
:101E9000BF90AF9008954F925F926F927F928F9212
:101EA0009F92AF92BF92CF92DF92EF92FF920F93E9
:101EB0001F93CF93DF938AEE94E48093C72090938F
:101EC000C82081E08093CF200E94645110EE412E03
:101ED0001BE2512EBCEC6B2EB7E07B2EA3EB8A2EBF
:101EE000A7E09A2EF4E6AF2EB12C4092DE2B509252
:101EF000DF2B0E943251AA2797FDA095BA2FBC0173
:101F0000CD0124ED30E340E050E00E94095C20E088
:101F100038E040E050E00E94715C79018A0184ED74
:101F200090E3A0E0B0E0E80EF91E0A1F1B1F670156
:101F300000D000D0CDB7DEB72196ADB7BEB71196B1
:101F40006D927C921297C801B70120E137E240E020
:101F500050E00E94715C2A833B83C701F7FE04C0F6
:101F6000882799278E199F0960E177E20E943C5CDF
:101F70008C839D830E941B5800D00F92CDB7DEB793
:101F80002196EDB7FEB781829282C801B701605AEF
:101F90007F408040904023EC30E040E050E00E94E1
:101FA000715C2A833B83C601805A9F4097FF03C020
:101FB000909581959F4F63EC70E00E943C5C9C0182
:101FC0002A9DC0012B9D900D3A9D900D112463EC2C
:101FD00070E00E943C5C6C837D83C801B701660F92
:101FE000771F881F991F6E0D7F1D801F911F605ED8
:101FF0007E428040904025E431E040E050E00E9485
:10200000715C205E3F4F2E833F83C601880F991F6E
:102010008C0D9D1D805E9E4297FF03C0909581951B
:102020009F4F65E471E00E943C5CDC01AA9DC00109
:10203000AB9D900DBA9D900D112465E471E00E9456
:102040003C5C688779870E941B58E091DE2BF091F9
:10205000DF2B1192E093DE2BF093DF2BEDB7FEB771
:102060003A96EDBFFEBF80E090E06FEE73E040E097
:1020700024E001E00E942546813009F036CF0E941D
:1020800029511092CF20DF91CF911F910F91FF9096
:10209000EF90DF90CF90BF90AF909F908F907F9008
:1020A0006F905F904F9008950F9384E094E06BE6FB
:1020B00072E045E020E101E00E942546823019F4FB
:1020C0000E94FE16F2CF833019F40E94F416EDCF71
:1020D000813059F70F910895CF92DF92EF92FF92DE
:1020E0000F931F93CF93DF930E94E75080EEC82E8B
:1020F0008BE2D82E01E0E02EF12CC092DE2BD092A4
:10210000DF2BC0E0D0E0C7010C2E02C0880F991F62
:102110000A94E2F70E94B15040E0811141E08FE360
:1021200093E060E10E946A452196C830D10559F7D5
:102130008FEF92E06BE672E047E022E101E00E945F
:102140002546813001F1182F12508FE393E06FEF95
:1021500072E0412F20E10E942546823049F4C701F8
:1021600002C0880F991F1A95E2F70E94B550C5CF9B
:10217000833019F6C70102C0880F991F1A95E2F73C
:102180000E94CF50BACFDF91CF911F910F91FF9056
:10219000EF90DF90CF9008958F929F92AF92BF9271
:1021A000CF92DF92EF92FF920F931F93DF93CF9323
:1021B000CDB7DEB72797CDBFDEBF81E08093CF20BC
:1021C0008AEE94E48093C7209093C82030EE832E4B
:1021D0003BE2932E5E010894A11CB11C2DEDC22E92
:1021E00027E0D22E90E6E92E96E0F92E1FE08092AD
:1021F000DE2B9092DF2BC5010E9419178DB79EB779
:102200000E978DBF9EBFEDB7FEB73196ADB7BEB787
:102210001196CD92DC92129789819A818283938361
:102220008B81848315828C81868317828D81808740
:1022300011868E81828713868F81848715860E94FE
:102240001B58E091DE2BF091DF2B1192E093DE2BF7
:10225000F093DF2BF70116838F818F7085838DB705
:102260009EB70E968DBF9EBF80E090E066E473E05F
:1022700040E024E001E00E942546813009F0B7CF1C
:102280001092CF202796CDBFDEBFCF91DF911F9157
:102290000F91FF90EF90DF90CF90BF90AF909F9005
:1022A0008F900895EF92FF920F931F93CF93DF9338
:1022B0000E940C0A0E9469160E94B34A40EEE42E66
:1022C0004BE2F42EC0E6D6E01FE0E092DE2BF09267
:1022D000DF2B8BE692E061E672E040E020E001E077
:1022E0000E942546813019F40E94CC104BC08230E8
:1022F00019F40E944B0F46C0833029F40E94F41653
:102300000E94FA4E3FC0843029F40E941A460E946F
:10231000DC1938C0853029F40E941A460E94BC5648
:1023200031C0863029F40E9454100E94F4162AC04D
:10233000873031F484E593E06BE672E046E01EC03E
:10234000883019F40E946C101DC0893019F40E9465
:10235000000C18C08A3019F40E94970E13C08B30FD
:1023600019F40E94E70D0EC08C3019F40E942E0C57
:1023700009C087EF95E06BE672E04CE024E001E0F5
:102380000E9425461E83A1CFFC018081807F862B81
:1023900080830895FC018081807F862B808308954F
:1023A000FC018181887F862B81830895FC018181D6
:1023B000887F862B81830895FC01838180718062F0
:1023C000862B83830895FC01838180718062862B34
:1023D00083830895FC018181607F862B818308952A
:1023E000FC0181816073862B81830895FC018181CA
:1023F000607F6095862381830895FC0181816073ED
:102400006095862381830895FC0186818C7F862BCD
:1024100086830895FC0186818C7F862B86830895B0
:10242000FC018681837F862B86830895FC0186814B
:10243000837F862B86830895FC0187818C7F862B82
:1024400087830895FC0187818C7F862B878308957D
:10245000FC018781837F862B87830895FC01878118
:10246000837F862B87830895FC0187818F7C862B51
:1024700087830895FC0187818F73862B8783089556
:10248000FC018081807F80838CE081870895FC013E
:102490008081807F80838CE081870895AF92CF9286
:1024A000EF920F93DC01FB016D937C9311971296D1
:1024B0004D935C93139714961C921497CC2011F4AF
:1024C00090E001C090E8222311F480E001C080E296
:1024D00000650A29902B892B8083ED91FC9111973F
:1024E000E18215961D921C9216971296ED91FC9121
:1024F000139780EA81830F91EF90CF90AF9008956A
:10250000EF920F93DC01FB016D937C931197129670
:102510004D935C931397222311F480E401C080E66D
:10252000802B8083ED91FC911197E1821296ED91C1
:10253000FC91139780E481830F91EF900895EF92BF
:102540000F931F93FC0100831183E28263837483E2
:10255000458356832783108611861F910F91EF9034
:102560000895CF93DF93DC011596CD91DC911697FA
:102570009885ED91FC911197808184FD05C081E0E3
:1025800014968C93149724C08381ED81FE81E90F0A
:10259000F11D80839F5F1596ED91FC9116978781C1
:1025A000981758F40380F481E02DE90FF11D808124
:1025B000ED91FC91119783830BC082810190F08192
:1025C000E02D85831596ED91FC91169781E081872A
:1025D0001596ED91FC9116979087DF91CF91089514
:1025E000CF93DF93DC01EB0114969C911497159621
:1025F000ED91FC911697309729F415966D937C9385
:10260000169710C08185882311F482E028C0992391
:1026100049F01296ED91FC911397848184FD02C0DC
:1026200081E01DC01596CD93DC93169719861496FC
:102630001C9214978A81E881F98186831596ED9121
:10264000FC91169710861596ED91FC9116970380D4
:10265000F481E02D8081ED91FC91838380E0DF9116
:10266000CF910895FC01A081B18113966C930190E4
:10267000F081E02D828187FFFDCF83810895CF9384
:10268000DF93EC01FB016115710511F480E037C0A7
:102690006D837E834281A081B181109711F01696DF
:1026A0004C93678190E01AC0292F30E00380F481B9
:1026B000E02DE20FF31F8081E881F9818383E881B7
:1026C000F981828187FFFDCF8381ED81FE810580C5
:1026D000F681E02DE20FF31F80839F5FED81FE8185
:1026E000961710F30190F081E02D309709F04583A3
:1026F000ED81FE816087ED81FE8181E08187DF9140
:10270000CF910895FC0181858C7F862B818742873C
:102710000895FC018185837F862B818743870895F7
:10272000EF920F93FC01442311F490E001C090E874
:10273000222311F480E001C080E4E02A9E29982B36
:102740008FB7F8946093B000908B8FBF0F91EF908C
:102750000895E0EBF0E09281907F982B92830895AA
:10276000E0EBF0E092819F70982B92830895E0EB6C
:10277000F0E09381907F982B93830895E0EBF0E055
:1027800093819F70982B938308950F93DF93CF933A
:102790000F92CDB7DEB72FB72983F8941BBEFC018B
:1027A00008ED04BF608389818FBF0F90CF91DF91C7
:1027B0000F910895662311F490E001C090E2482B38
:1027C000942BE0E5F0E0928308956F71682BE0E5CB
:1027D000F0E065830895E0E5F0E02081982F909582
:1027E000922390839081892308950F93DF93CF9351
:1027F0000F92CDB7DEB79FB79983F8941BBE682BB5
:1028000081E490E0FC0108ED04BF608389818FBF03
:102810000F90CF91DF910F9108950F93DF93CF9396
:102820000F92CDB7DEB7209140009FB79983F894FF
:102830001BBEA0E4B0E0287F282BFD0108ED04BFFB
:10284000208399819FBF9C9189230F90CF91DF9125
:102850000F910895E0E4F0E09381917F9160982BCF
:1028600093830895282F30915600662311F0982FF6
:1028700001C090E0822F80958323982BE0E5F0E063
:102880009683213031F480916800816080936800E4
:102890000895223029F48091600081608093600067
:1028A00008950F93DF93CF930F92CDB7DEB78FB715
:1028B0008983F8941BBE23E083E590E0FC0108EDDA
:1028C00004BF208389818FBF0F90CF91DF910F913B
:1028D00008950F93DF93CF930F92CDB7DEB78FB7E5
:1028E0008983F8941BBE21E082E490E0FC0108EDAE
:1028F00004BF208389818FBF0F90CF91DF910F910B
:1029000008950197E0E0F4E08287938760877187FC
:10291000448755878081887F822B80830895E0E0FB
:10292000F4E092819C7F982B92830895E0E0F4E09C
:102930009281937F982B92830895E0E0F4E0928156
:10294000907F982B962B92830895209108043091C4
:102950000904280F391F80910A0490910B048217F3
:10296000930730F480910A0490910B04281B390BD3
:10297000E0E0F4E0248735870895E0E0F4E090811A
:10298000987F982B90830895FC0160837183428324
:10299000EC5FFE4F108212923396108212920895CD
:1029A000FC0162830895FC01EB5FFE4F81919081F1
:1029B00020E08F5F8F77891321E0822F0895CF93D6
:1029C000DF93DC01EC01CB5FDE4F8881AA5FBE4F55
:1029D0009C91A650B14020E08F5F8F778917A1F0BE
:1029E00021E08881FD01E80FF11DED57FF4F608365
:1029F0008F5F8F778883ED91FC91119783818C7F16
:102A000012969C91892B8383822FDF91CF91089519
:102A1000FC01ED5FFE4F9191808120E0981321E051
:102A2000822F0895FC01DC01AC5FBE4F8C91E80F52
:102A3000F11D83819C919F5F9F779C930895CF9315
:102A4000DF93DC01EC01CD5FDE4F98819F5F9F77C4
:102A5000AC5FBE4F8C91A450B140ED91FC911197A9
:102A6000E081981711F480E007C08881A80FB11D9C
:102A70001396EC93988381E0DF91CF910895CF93E3
:102A8000DF93FC01EC01CA5FDE4F9881EB5FFE4FE4
:102A90008081E550F140A081B181891739F4139606
:102AA0008C9113978C7F13968C930BC08881E80FC1
:102AB000F11DED57FF4F80818C9388818F5F8F7759
:102AC0008883DF91CF910895FC0170FF03C084815A
:102AD000816002C084818E7F848360830895FC01BD
:102AE000848180FF05C08081282F30E0316003C0E1
:102AF0008081282F30E0C901089580918000836093
:102B000098ED94BF809380008091820080FDFCCF7F
:102B10000895836098ED94BF809380008091820037
:102B200080FDFCCF0895E0E8F0E080818C7F81603B
:102B300098ED94BF80830895E0E8F0E08181869568
:102B4000817008952091800090918100936088EDBC
:102B500084BFE0E8F0E091838091820080FDFCCFAB
:102B60002695822F8170089520918000836098EDD2
:102B700094BFE0E8F0E081838091820080FDFCCF8B
:102B80002695822F81700895E0E8F0E081818C7FA6
:102B9000816098ED94BF818308951F920F920FB6C4
:102BA0000F9208B60F9209B60F920BB60F9211242E
:102BB00018BE19BE1BBE2F933F934F935F936F9325
:102BC0007F938F939F93AF93BF93EF93FF9382E590
:102BD00091E20E943F15FF91EF91BF91AF919F91BC
:102BE0008F917F916F915F914F913F912F910F90B6
:102BF0000BBE0F9009BE0F9008BE0F900FBE0F9036
:102C00001F9018951F920F920FB60F9208B60F9251
:102C100009B60F920BB60F92112418BE19BE1BBE37
:102C20002F933F934F935F936F937F938F939F93D4
:102C3000AF93BF93EF93FF9382E591E20E941F153C
:102C4000FF91EF91BF91AF919F918F917F916F9184
:102C50005F914F913F912F910F900BBE0F9009BE46
:102C60000F9008BE0F900FBE0F901F90189582E531
:102C700091E20E9408158823D1F382E591E20E9437
:102C8000121508951F93182F82E591E2612F0E947B
:102C9000DF148823C9F31F910895EF920F93E091F9
:102CA0005221F091532184818F7E84838481877F98
:102CB000848388E0E0EAF6E0828380EA96E068E0D8
:102CC00040E020E000E0EE240E9490130F91EF908E
:102CD0000895EF920F93E0EAF6E088E08583818320
:102CE00084E0828380EA96E064E040E020E008E14E
:102CF000EE240E94901382E591E260EA7BE041E0DD
:102D00000E94C414E0915221F091532183E0858305
:102D100083818F7C80618383A0EABBE081E016968B
:102D20008C93169717961C9284818061848384818A
:102D300088608483E0EAF0E08281816082830F9181
:102D4000EF9008951F920F920FB60F9208B60F9250
:102D50000BB60F92112418BE1BBE8F939F93EF9357
:102D6000FF939091D9229230A1F0933028F49923C7
:102D7000E1F0913001F507C0943089F0943048F0CB
:102D80009530C9F412C0E0E6F6E082E0878384E083
:102D900011C0E0E6F6E084E0878388E00BC0E0E65F
:102DA000F6E082E08783978306C0E0E6F6E081E004
:102DB000878382E087838091D922853019F410922D
:102DC000D92205C08091D9228F5F8093D922FF91AB
:102DD000EF919F918F910F900BBE0F9008BE0F90B7
:102DE0000FBE0F901F90189580E498E060E00E945D
:102DF000CA118FE0E0E6F6E0868308951092D922AA
:102E0000E0E6F6E08FE0868381E08583E0E4F8E0A9
:102E100088E081878AE196E086A397A380E498E022
:102E200061E00E940A1280E498E067E00E94CA1103
:102E30000895FC01F8948091DB229091DC2280833C
:102E400091838091DD2282838091DE228383809131
:102E5000DF2284838091E02285838091E122868332
:102E6000789481E008959091E1228091DA22891787
:102E700011F480E008958091E1228093DA2281E0CC
:102E80000895FC01F894808191818093DB229093D6
:102E9000DC2282818093DD2283818093DE22848103
:102EA0008093DF2285818093E02286818093E122D6
:102EB000789481E00895F8948AED97E08093DB227E
:102EC0009093DC2281E08093DD228093DE221092B9
:102ED000DF221092E0221092E1221092DA227894FE
:102EE00008959C0164E670E00E94285C892B31F40F
:102EF000C90160E971E00E94285C0895822F837007
:102F000008951F920F920FB60F9208B60F9209B64E
:102F10000F920BB60F92112418BE19BE1BBE2F9331
:102F20003F934F935F936F937F938F939F93AF9351
:102F3000BF93EF93FF938091E1228F5F8093E12213
:102F40008091E1228C3309F069C01092E1228091D6
:102F5000E0228F5F8093E0228091E0228C3309F0A1
:102F60005DC01092E0228091DF228F5F8093DF228C
:102F70008091DF22883109F051C01092DF228091C8
:102F8000DE228F5F8093DE228091DE22803271F11B
:102F90008091DE228F3189F48091DD22843031F1FD
:102FA0008091DD22863011F18091DD228930F1F0AF
:102FB0008091DD228B3011F519C08091DE228E3197
:102FC00029F48091DD228230C9F410C08091DE2284
:102FD0008D31A1F48091DD22823081F48091DB2259
:102FE0009091DC220E947117882341F08091DD22AC
:102FF0008F5F8093DD2281E08093DE228091DD224D
:103000008D3061F481E08093DD228091DB2290910C
:10301000DC2201968093DB229093DC22FF91EF91DA
:10302000BF91AF919F918F917F916F915F914F91E0
:103030003F912F910F900BBE0F9009BE0F9008BECD
:103040000F900FBE0F901F90189500001895BF921B
:10305000CF92DF92EF92FF920F931F93CF93DF9364
:10306000182F092FB22E00D000D08DE89FE0ADB709
:10307000BEB711968D939C931297EDB7FEB743831D
:103080005483658376830E941B58212F302FC901FA
:10309000EC017C0110E08DB79EB706968DBF9EBFF8
:1030A00087E8C82E8FE0D82E17C000D00F92EDB75A
:1030B000FEB73196ADB7BEB71196CD92DC9212979E
:1030C000D7018D917D01828313820E941B581F5F5F
:1030D0000F900F900F900F901B1538F380E20E9415
:1030E000CA5710E00CC09881892F80528F3510F09C
:1030F0008EE201C0892F0E94CA571F5F21961B15BF
:1031000090F38AE00E94CA57DF91CF911F910F91EF
:10311000FF90EF90DF90CF90BF900895482F21EA65
:103120003FE090E007C0F9012F5F3F4FE491EE23AD
:10313000D1F79F5F941721F0F9018491882399F7C3
:1031400000D000D0EDB7FEB7319684E99FE0ADB76F
:10315000BEB711968D939C9312974283138224835A
:1031600035830E941B58EDB7FEB73696EDBFFEBF04
:103170000895DF93CF93CDB7DEB72797CDBFDEBFDE
:10318000CE0101960E9419172C8130E040E050E0FA
:10319000A901332722278B8190E0A0E0B0E0F5E180
:1031A000880F991FAA1FBB1FFA95D1F7282B392B1F
:1031B0004A2B5B2B8D8190E0A0E0B0E0EBE0880F24
:1031C000991FAA1FBB1FEA95D1F7282B392B4A2B31
:1031D0005B2B8E8190E0A0E0B0E075E0880F991F36
:1031E000AA1FBB1F7A95D1F7282B392B4A2B5B2BB3
:1031F0008F81869590E0A0E0B0E0282B392B4A2BF8
:103200005B2B89819A818C5B9740A0E0B0E069E1FB
:10321000880F991FAA1FBB1F6A95D1F7282B392B3E
:103220004A2B5B2BB901CA012796CDBFDEBFCF91D8
:10323000DF910895EF92FF920F931F93CF93DF9347
:103240007C018B01C0E0D0E0015010400E94371695
:103250008D3099F0883021F42097C1F321970AC06E
:103260008032A0F3C017D1078CF7F701EC0FFD1FD8
:10327000808321960E944216E9CFCE0DDF1D188271
:103280008DE00E9442168AE00E944216DF91CF91A3
:103290001F910F91FF90EF9008959F92AF92BF9270
:1032A000CF92DF92EF92FF920F931F93DF93CF9312
:1032B000CDB7DEB76697CDBFDEBF8C017E01089427
:1032C000E11CF11CC701B8010E94C43D882309F02C
:1032D00064C0D8010D900020E9F71197A01BB10B35
:1032E00057016801CA0EDB1E8FE2982E7D010894FB
:1032F000E11CF11CE00EF11E44C09E3209F441C0F5
:1033000080914E2784FF18C080915C2790915D27A3
:10331000019680935C2790935D27F6019082C70108
:103320006FE477E20E94BF5CC8010E944D19F6016C
:103330001082882331F131C080915E2790915F2700
:10334000019680935E2790935F278091622B9091E6
:10335000632BA091642BB091652B2091462730916F
:1033600047274091482750914927820F931FA41F58
:10337000B51F8093622B9093632BA093642BB09323
:10338000652BC50166E477E20E94672F882329F444
:1033900090914F27992309F0B0CF6696CDBFDEBF3D
:1033A000CF91DF911F910F91FF90EF90DF90CF9021
:1033B000BF90AF909F9008952F923F924F925F924F
:1033C0006F927F928F929F92AF92BF92CF92DF9235
:1033D000EF92FF920F931F93DF93CF93CDB7DEB79A
:1033E000C657D040CDBFDEBFE0E4F9E088E081877A
:1033F00080E49CE986A397A380E499E061E00E94C1
:103400000A1280E499E064E00E94CA1182E496E125
:103410008093C7209093C82081E69FE00E94D957EF
:1034200080E49FE00E94D95784E29FE00E94D95730
:1034300044245524320156E6252E5BE2352E8EE3D8
:103440000E94CA5786E69BE268E770E00E941A195C
:103450008091662B47E6A42E4BE2B42EAA82BB8253
:10346000863609F444C3873630F4823609F4E4C161
:10347000843629F70CC0843711F40C945223883712
:1034800011F40C94BD238836D1F60C94E42380917A
:10349000672B28E63BE22A833B83893609F47BC00D
:1034A000833709F49DC0843651F68E010E5F1F4F9D
:1034B000C801BE01625F7F4F0E947958882309F4DA
:1034C000BECFC801BE016E5E7F4F0E94795888232F
:1034D00021F44A8A5B8A6C8A7D8A32E6E32E37E2DF
:1034E000F32E2A893B894C895D898E85B70101E0DD
:1034F0000E941C41882351F000D00F92EDB7FEB717
:1035000031962DE1A22E2FE0B22E5BC0AA88BB8897
:10351000CC88DD8800D000D0E1E1FFE0ADB7BEB7D8
:103520001196ED93FC9312971396AD92BD92CD92A6
:10353000DC9216970E941B58EA82FB82EE24FF243D
:103540008701EDB7FEB73696EDBFFEBF8A819B813E
:10355000B801A70120E10E9427188A819B8140962B
:103560008A839B8380E190E0A0E0B0E0E80EF91E42
:103570000A1F1B1F90E0E91692E0F90690E0090788
:1035800090E0190719F7250136010894411C511CD8
:10359000611C711C54CFCE010296BE01625F7F4F49
:1035A0000E947958882309F44ACF8E850E94C94326
:1035B00000D00F92EDB7FEB731969AE0A92E9FE0AA
:1035C000B92EADB7BEB71196AD92BC921297828359
:1035D00013820E941B580F900F900F900F902FCFC7
:1035E000CE010296BE01625F7F4F0E947958882308
:1035F00009F425CF8E8561E0AE014E5E5F4F0E94DB
:103600006F418823E1F400D000D0E1EFFEE0ADB7D8
:10361000BEB71196ED93FC9312978A899B89AC896A
:10362000BD89EDB7FEB783839483A583B6830E94DB
:103630001B582DB73EB72A5F3F4F2DBF3EBF8E852B
:1036400062E0AE014C5F5F4F0E946F418823B1F48E
:1036500000D00F92E0EEFEE0ADB7BEB71196ED934D
:10366000FC9312978C819D8113968D939C93149754
:103670000E941B580F900F900F900F908E8563E063
:10368000AE014E5E5F4F0E946F418823E1F400D08F
:1036900000D0E1ECFEE0ADB7BEB71196ED93FC9320
:1036A00012978A899B89AC89BD89EDB7FEB7838360
:1036B0009483A583B6830E941B582DB73EB72A5F1B
:1036C0003F4F2DBF3EBF8E856AE0AE014F5F5F4F1B
:1036D0000E946F418823C1F400D00F92EDB7FEB76E
:1036E000319602EBA02E0EE0B02EADB7BEB711960C
:1036F000AD92BC9212978981828313820E941B58DB
:103700000F900F900F900F908E856BE042E657E27E
:103710000E946F41882369F48CEA9EE00E94D95789
:1037200082E697E240E050E060E070E020E10E9435
:1037300027188E856CE042E657E20E946F4188238D
:1037400069F486EA9EE00E94D95782E697E240E05B
:1037500050E060E070E020E10E9427188E856DE067
:1037600042E657E20E946F41882369F480EA9EE0B6
:103770000E94D95782E697E240E050E060E070E0B6
:1037800024E00E9427188E856EE042E657E20E94F0
:103790006F418823C9F484E99EE00E94D9571E82B4
:1037A0001F820DC0AC0160E070E08E59984D20E1A1
:1037B0000E9427188E819F8140968E839F838E81E1
:1037C0009F818034910570F38E8565E146E65BE26A
:1037D0000E946F418823B1F410928E2B00D00F927B
:1037E000E9E8FEE0ADB7BEB71196ED93FC931297F2
:1037F00013962D923C9214970E941B580F900F9095
:103800000F900F908E8566E146E65BE20E946F4165
:10381000882309F014CE10927A2B00D00F92E0E8A2
:10382000FEE0ADB7BEB71196ED93FC9312971396D9
:103830002D923C921497CDCE8091672B18E6A12E45
:103840001BE2B12EAA82BB82863609F43DC18736BF
:1038500030F4843659F0853609F0F1CD3EC0823718
:1038600009F4C0C0873709F0EACDF5C0CE01029651
:10387000BE01625F7F4F0E947958882309F4DFCD33
:103880008E859F858E59984D8A839B83EE84FF8415
:103890000889198980E290E08A879B8719C08A810C
:1038A0009B81B801A70120E10E9427188A859B858A
:1038B00001978A879B878A819B8140968A839B8315
:1038C00080E190E0A0E0B0E0E80EF91E0A1F1B1FA7
:1038D0008A859B85892B19F7B2CD8E010E5F1F4F0C
:1038E000C801BE01625F7F4F0E947958882309F4A6
:1038F000A6CDB2E1EB2EF12CEC0EFD1EC801B701F6
:103900000E9479588823C9F0680187018E859F85B8
:10391000A889B989FC01EE59F84D2A8920830196BE
:10392000A11DB11D8E879F87A88BB98BC601B801D9
:103930000E947958882351F782CD680187012E852E
:103940003F854889598900D000D0EDB7FEB7319640
:10395000A5E7AA2EAEE0BA2EADB7BEB71196AD92CE
:10396000BC92129722833383C9018E59984DDC0192
:103970008C91848315820E941B58EDB7FEB7369652
:10398000EDBFFEBF86E69BE268E770E00E941A1971
:103990002A823B828091662B8E3209F450CD803290
:1039A00028F48E859F85A889B9890FC0C601B80102
:1039B0000E947958882389F08E859F85A889B989C6
:1039C000FC01EE59F84D2A8920830196A11DB11DF5
:1039D0008E879F87A88BB98BB2CF80E79EE00E942D
:1039E000D957ADCF8E010E5F1F4FC801BE01625F78
:1039F0007F4F0E947958882309F421CDC801BE0168
:103A00006E5E7F4F0E947958882309F418CDC80153
:103A1000BE016A5E7F4F0E947958882341F481E09D
:103A200090E0A0E0B0E08E8B9F8BA88FB98F2A89A1
:103A30003B894C895D898E8562E677E20E890E941A
:103A40001C4100D00F92EDB7FEB7319679E6A72E54
:103A50007EE0B72EB6CD8E010E5F1F4FC801BE01AE
:103A6000625F7F4F0E947958882309F4E8CCC8012F
:103A7000BE016E5E7F4F0E947958882309F4DFCC27
:103A8000C801BE016A5E7F4F0E947958882341F4C5
:103A900081E090E0A0E0B0E08E8B9F8BA88FB98F83
:103AA0002A893B894C895D898E8562E677E20E8999
:103AB0000E945B4300D00F92EDB7FEB7319662E6ED
:103AC000A62E6EE0B62E7DCDCE010296BE01625FBF
:103AD0007F4F0E947958882309F4B1CC6E8582E625
:103AE00097E270E040E054E00E94AD5CA8CC809189
:103AF000672B28E63BE22A833B8390E0FC01E156FA
:103B0000F040E831F10508F09ACCE650FF4FEE0F97
:103B1000FF1F0590F491E02D1994CE010296BE018D
:103B2000625F7F4F0E947958882309F488CC8E8584
:103B30009F85A889B98922E332E0829FB001839FE3
:103B4000700D929F700D11246E517D4D0E945F2566
:103B5000A5C588E69BE2BE016E5E7F4FAE01445F65
:103B60005F4F0E945F3C882309F098C52C853D85F6
:103B70008DB79EB780978DBF9EBFEDB7FEB73196CC
:103B80008BE99DE0ADB7BEB711968D939C931297CC
:103B9000D9018C918283138212968C9190E0A0E0DF
:103BA000B0E059E0880F991FAA1FBB1F5A95D1F7A3
:103BB00084839583A683B783D90113968C91139739
:103BC0008087118618968D919C911997828793878B
:103BD0005A964D915D916D917C915D974487558783
:103BE000668777875E964D915D916D917C919197F7
:103BF0004250504060407040408B518B628B738BC1
:103C000092964D915D916D917C919597448B558BDA
:103C1000668B778B96964D915D916D917C9199977E
:103C2000408F518F628F738F9A962D913D914D9158
:103C30005C919D97248F358F468F578F0E941B581C
:103C400010925C2710925D2710925E2710925F27DA
:103C50001092622B1092632B1092642B1092652BA2
:103C6000EDB7FEB7B096EDBFFEBF8A819B810E9483
:103C70004D19882309F012C5EC85FD85E280E69494
:103C80002DB73EB7225130402DBF3EBFCDB6DEB678
:103C90000894C11CD11C8DE49DE0ADB7BEB7119650
:103CA0008D939C93129780915E2790915F27D60108
:103CB00012968D939C9313972091622B3091632BD6
:103CC0004091642B5091652B14962D933D934D9309
:103CD0005C93179780915C2790915D2718968D9340
:103CE0009C931997FF2400E010E0268D378D40A1AA
:103CF00051A12250304040405040C801B7010E94BD
:103D0000095CF60162877387848795872A893B89D6
:103D10004C895D89C801B7010E94095CD6011E96D5
:103D20006D937D938D939C9351970E941B58EDB793
:103D3000FEB772967EC18E010F5D1F4FC80168E607
:103D40007BE20E94C43D882309F0A8C41886198626
:103D50001E821F821E861F86188A198A6801C60164
:103D600066E477E20E94672F882309F0B5C080914E
:103D70004F27882309F4B0C080914E2784FF06C0E6
:103D80008885998501968887998719C08E819F813A
:103D900001968E839F838E859F85A889B9892091FE
:103DA0004627309147274091482750914927820F55
:103DB000931FA41FB51F8E879F87A88BB98B8091F7
:103DC0004E2784FD04C04DE2E42EF12C03C034E400
:103DD000E32EF12C80FD03C00DE210E002C002E5ED
:103DE00010E081FD04C02DE2822E912C03C098E4E6
:103DF000892E912C82FD03C06DE270E002C063E564
:103E000070E085FD03C08DE290E002C081E490E0A7
:103E100020914A2730914B2740914C2750914D27B4
:103E2000ADB7BEB75C97ADBFBEBFEDB7FEB73196BD
:103E30000F2EF2E2AF2EFDE0BF2EF02D1196AD92C7
:103E4000BC921297E282F382048315838682978262
:103E50006087718782879387C901892F9927869503
:103E60008454984F84879587C90165E09695879516
:103E70006A95E1F78F709070868797872F71307001
:103E8000208B318B852F869586958695828B138A1C
:103E900005E0569547950A95E1F74F735070448BAE
:103EA000558B8091462790914727A0914827B09144
:103EB0004927868B978BA08FB18F2FE437E2228F13
:103EC000338F0E941B588DB79EB74C968DBF9EBFF7
:103ED0008AE00E94CA5743CFADB7BEB71A97ADBFAD
:103EE000BEBFEDB7FEB7319689EF9CE011968D937A
:103EF0009C9312978E819F81828393838E859F8569
:103F0000A889B98984839583A683B7838885998591
:103F1000808791870E941B58EDB7FEB73A96EDBF98
:103F2000FEBF8A819B81BE01625F7F4FAE01445F0D
:103F30005F4F0E945F3C882309F081CA00D000D007
:103F400084EE9CE0ADB7BEB711968D939C9312970B
:103F5000EC85FD85628170E080E090E02E853F85F4
:103F6000488959890E94095C22E030E040E050E035
:103F70000E94715CEDB7FEB723833483458356837B
:103F80000E941B582DB73EB72A5F3F4FF2C3CE01A8
:103F90000296BE01625F7F4F0E947958882309F420
:103FA0004ECA6A817B81CE01C7964E850E94903EA3
:103FB00075C3CE01C7960E94193270C3CE01029616
:103FC000BE01625F7F4F0E947958882309F437CA87
:103FD0004E855F8568897989CE01C7960E94B22F88
:103FE000182F0E948E18112309F029CAFE01FD9690
:103FF00020813181428153818DB79EB70A978DBF51
:104000009EBFEDB7FEB7319681ED9CE0ADB7BEB770
:1040100011968D939C931297228333834483558307
:1040200026833783408751870E941B58EDB7FEB720
:104030003A96EDBFFEBF03CACE010296BE01625F93
:104040007F4F0E947958882309F4F9C91A8A1B8A7C
:104050001C8A1D8A1092602710926127C12C14E0DF
:10406000D12EB7E3EB2EF12CEC0EFD1E8E01085F76
:104070001F4F3CC08030F4E09F07F0E0AF07F0E056
:10408000BF075CF0CA86DB8680509440A040B040F9
:104090008E879F87A88BB98B06C08A879B871E86D1
:1040A0001F86188A198A4A855B85C70162E677E20E
:1040B00098010E94FE33882319F00E948E181FC0B9
:1040C000688579859B0140E050E08A899B89AC89AD
:1040D000BD89820F931FA41FB51F8A8B9B8BAC8B4E
:1040E000BD8B8A859B858617970749F48E859F85AA
:1040F000A889B9890097A105B10509F0BBCFE09067
:104100006027F0906127E886F9866A897B898C8927
:104110009D892DB73EB72A5030402DBF3EBFCDB64A
:10412000DEB60894C11CD11C2DEA3CE0E8C0CE01EB
:104130000296BE01625F7F4F0E947958882309F47E
:104140007EC9FE01FD96E080F18002811381A0E12D
:104150008A2E912CF7E3AF2EB12CAC0EBD1EEAE0F7
:10416000CE2ED12CCC0EDD1E34C080319105A105A0
:10417000B10554F08A869B864097A109B1098E87C4
:104180009F87A88BB98B06C08A879B871E861F8650
:10419000188A198A4A855B85C50162E677E296012D
:1041A0000E94FE33882309F079C22A853B852115B8
:1041B000310509F444C982E697E2B801A7010E94DB
:1041C000271880E190E0A0E0B0E0E80EF91E0A1F99
:1041D0001B1F8E859F85A889B9890097A105B10508
:1041E00021F62DC98E010E5F1F4FC801BE01625F0F
:1041F0007F4F0E947958882309F421C9C801BE0164
:104200006E5E7F4F0E947958882309F418C96A8925
:1042100082E697E270E040E054E00E94AD5C1A8ACA
:104220001B8A1C8A1D8A1092602710926127C12C5C
:1042300074E0D72E67E3E62EF12CEC0EFD1E8E0106
:10424000085F1F4F3CC08030E4E09E07E0E0AE070F
:10425000E0E0BE075CF0CA86DB8680509440A04058
:10426000B0408E879F87A88BB98B06C08A879B87B3
:104270001E861F86188A198A4A855B85C70162E6F1
:1042800077E298010E942532882319F00E948E1847
:104290001FC0688579859B0140E050E08A899B8931
:1042A000AC89BD89820F931FA41FB51F8A8B9B8B7E
:1042B000AC8BBD8B8A859B858617970749F48E85C5
:1042C0009F85A889B9890097A105B10509F0BBCFE1
:1042D000E0906027F0906127E886F9866A897B89FB
:1042E0008C899D892DB73EB72A5030402DBF3EBFE7
:1042F000CDB6DEB60894C11CD11C26E83CE0ADB7B3
:10430000BEB711962D933C931297F6016283738387
:104310008483958324E630E040E050E00E94095C0D
:1043200000E010E0A80197010E94715CD60116968A
:104330002D933D934D935C93199776CECE01C796FE
:104340000E94DA2EABC188E69BE260E270E00E9438
:10435000B45CFC01009709F472C811928A819B81B8
:10436000BF010E9461389AC188E69BE20E94BF3B70
:1043700095C188E69BE20E942B3A90C18E010E5FA8
:104380001F4FC801BE01625F7F4F0E94795888238A
:1043900009F455C8C801BE016E5E7F4F0E9479586E
:1043A000882309F44CC88A819B816E854A890E94C2
:1043B000E13974C18E010E5F1F4F5EE0A52EB12C56
:1043C000AC0EBD1EC801B5010E947958882309F4BE
:1043D00036C842E1C42ED12CCC0EDD1EC801B60178
:1043E0000E947958882309F42AC836E1E32EF12C7B
:1043F000EC0EFD1EC801B7010E947958882309F40C
:104400001EC88E859F85A889B9898C5B9740A0407E
:10441000B04029E0880F991FAA1FBB1F2A95D1F72A
:104420002A893B894C895D892F70307040705070AB
:10443000F5E0220F331F441F551FFA95D1F7822B49
:10444000932B2E893F892F713070822B932B809371
:104450004A2790934B27C801B5010E9479588823B9
:1044600011F40C941F1AC801B6010E9479588823D0
:1044700011F40C941F1AC801B7010E9479588823BF
:1044800011F40C941F1A8A899B89AC89BD898F739A
:104490009070A070B070E5E0880F991FAA1FBB1F35
:1044A000EA95D1F72E893F89488D598D55954795C5
:1044B000379527952F713070282B392B8E859F8546
:1044C000A889B9896BE0880F991FAA1FBB1F6A953D
:1044D000D1F7282B392B20934C2730934D278A81F5
:1044E0009B8166E477E20E948F39D8C088E69BE220
:1044F00060E270E00E94B45C8C01009711F40C94AF
:104500001F1ADC011C9200D00F9259E7A52E5CE027
:10451000B52EEDB7FEB7A182B2828A819B818383DB
:1045200094830E941B580F900F900F900F9047E3B9
:10453000E42EF12CEC0EFD1E6A817B81C70141E067
:104540000E94903E882309F0A9C00F5F1F4F00D042
:104550000F92EAE6FCE0ADB7BEB71196ED93FC937F
:10456000129713960D931C9314970E941B580F904B
:104570000F900F900F90CE01895A9F4FB8014AE0DB
:104580000E94903E882321F00E948E18C7016FC0C0
:104590000F920F928EE59CE0ADB7BEB711968D934A
:1045A0009C9312970E941B581E861F86188A198A90
:1045B0000F900F90670136E0E32EF12CEC0EFD1EFC
:1045C0008E01085F1F4FC60162E677E240E054E0CB
:1045D00097010E94FE33682F882339F54E815F8151
:1045E0004115510529F1CE01895A9F4F62E677E2C4
:1045F00098010E942532682FE885F9859F0140E0E7
:1046000050E08E859F85A889B989820F931FA41FCA
:10461000B51F8E879F87A88BB98B662331F48E8157
:104620009F81E817F90778F603C0862F0E948E183D
:1046300000D000D08AE49CE0EDB7FEB7818392837E
:104640008E859F85A889B98983839483A583B68342
:104650000E941B582DB73EB72A5F3F4F2DBF3EBF6C
:10466000CE01C7960E941932CE01895A9F4F0E94EF
:1046700019320C941F1A88E69BE20E94273E0EC056
:10468000CE010296BE01625F7F4F0E947958882357
:1046900011F40C941F1A8E850E9474250E948E18A6
:1046A0000C941F1A8E010E5F1F4F2EE0E22EF12C8C
:1046B000EC0EFD1EC801B7010E947958882351F104
:1046C0008E859F858A8F9B8FC801B7010E9479587C
:1046D0008E858C8FC801B7010E9479588E858D8F89
:1046E000C801B7010E9479588E858E8FC801B70125
:1046F0000E9479588E858F8FC801B7010E94795822
:10470000882311F40C941F1A8E8588A3CE014A9633
:104710000E944117CE014A960E9419178DB79EB785
:104720000E978DBF9EBFEDB7FEB7319691E3A92ED0
:104730009CE0B92EADB7BEB71196AD92BC92129760
:104740008A8D9B8D828393838C8D848315828D8D3E
:10475000868317828E8D808711868F8D8287138640
:1047600088A1848715860E941B582DB73EB7225F0B
:104770003F4F2DBF3EBF0C941F1ACE01C7960E941B
:10478000193280E060E070E00E945F2580E499E0EB
:1047900060E00E94CA1180E090E0CA58DF4FCDBFB0
:1047A000DEBFCF91DF911F910F91FF90EF90DF90CF
:1047B000CF90BF90AF909F908F907F906F905F90C1
:1047C0004F903F902F90089589E09CE00E94D95728
:1047D00088EE9BE00E94D95786EC9BE00E94D95757
:1047E00089EA9BE00E94D9578FE79BE00E94D95746
:1047F00085E49BE00E94D9578AE09BE00E94D9574C
:104800008CEE9AE00E94D95782EC9AE00E94D95728
:1048100089E99AE00E94D95788E79AE00E94D9571F
:1048200084E49AE00E94D95781E39AE00E94D95724
:104830008EE09AE00E94D95788EF99E00E94D957FC
:1048400089EC99E00E94D9578CEA99E00E94D957E7
:1048500088E999E00E94D95787E699E00E94D957E4
:1048600085E499E00E94D95785E299E00E94D957E2
:1048700080EF98E00E94D9578DEB98E00E94D957BD
:1048800087E998E00E94D95781E798E00E94D957BC
:104890008DE498E00E94D9578AE098E00E94D957A9
:1048A00080E098E00E94D95786EF97E00E94D957A0
:1048B0000C941F1A1F920F920FB60F9208B60F9208
:1048C00009B60F920BB60F92112418BE19BE1BBE6B
:1048D0002F933F934F935F936F937F938F939F9308
:1048E000AF93BF93EF93FF938091602790916127DF
:1048F000019680936027909361270E940C40FF915E
:10490000EF91BF91AF919F918F917F916F915F9147
:104910004F913F912F910F900BBE0F9009BE0F90BA
:1049200008BE0F900FBE0F901F901895EF92FF9248
:104930000F931F93CF93DF93EC017A018B018EEFDE
:104940009FEFAFEFBFEFE80EF91E0A1F1B1F8E8D02
:104950009F8DA8A1B9A10297A109B109E816F9068E
:104960000A071B0728F020E030E040E050E012C0CA
:104970002A8130E040E050E0C801B7010E94095CA4
:104980009B01AC018AA59BA5ACA5BDA5280F391F2D
:104990004A1F5B1FB901CA01DF91CF911F910F918F
:1049A000FF90EF900895EF92FF920F931F93CF9394
:1049B000DF93FC017B01EB01299686859785A08911
:1049C000B1890097A105B10509F471C062897389A5
:1049D00080E090E0FB01E80FF91FE081E03241F058
:1049E000E53009F4E5EEE99301968830910591F7F9
:1049F000DB0118968C91803211F48E0112C08EE288
:104A0000FE0181938F01FB019E012C5F3F4F80854A
:104A1000803239F0D8018D938D013196A217B307FA
:104A2000B1F7FB018385D70118968C93278D30E071
:104A300040E050E0522F442733272227868D90E014
:104A4000A0E0B0E0DC0199278827282B392B4A2BDE
:104A50005B2B848D90E0A0E0B0E0282B392B4A2B13
:104A60005B2B958D80E0A0E0B0E0282B392B4A2B02
:104A70005B2BF7012083318342835383DB015996FB
:104A80009C91599780E058962C91589730E0822B52
:104A9000932B8483958357969C91579780E05696E5
:104AA0002C9130E0822B932B86839783E801188228
:104AB000DF91CF911F910F91FF90EF900895DB014F
:104AC000882311F08BE00895E091B620F091B72093
:104AD000309709F01082109709F01C92A093B6202D
:104AE000B093B72080E00895882311F08BE00895FB
:104AF0001092BA2080E008956F927F928F929F92D9
:104B0000AF92BF92CF92DF92EF92FF920F931F93DB
:104B1000CF93DF93EC014A015B01CEA4DFA4E8A8A8
:104B2000F9A8C416D506E606F70609F44EC08C812E
:104B30008823A1F192E3692E712C6C0E7D1E898170
:104B4000B301A701960101E00E945B438823D9F5D8
:104B50001C828A8D9B8DAC8DBD8D2AA13BA14CA161
:104B60005DA1820F931FA41FB51FC816D906EA06C0
:104B7000FB06A0F41B8110C08A8D9B8DAC8DBD8D72
:104B8000C80ED91EEA1EFB1E8981B301A70196013A
:104B900001E00E945B431150123070F781149104C0
:104BA000A104B10491F0BE016E5C7F4F8981A50123
:104BB000940101E00E941C41882329F48EA69FA63F
:104BC000A8AAB9AA03C081E001C080E0DF91CF911B
:104BD0001F910F91FF90EF90DF90CF90BF90AF901B
:104BE0009F908F907F906F9008952F923F924F9259
:104BF0005F926F927F928F929F92AF92BF92CF926D
:104C0000DF92EF92FF920F931F93CF93DF933C01BC
:104C10006A017B0148015901423051056105710566
:104C200008F4BAC0F301868D978DA0A1B1A14817F1
:104C300059076A077B0708F0AFC022A033A044A041
:104C400055A08081823009F464C0833009F47AC0B1
:104C5000813011F022E09CC0EA01D695C795C40FBF
:104C6000D51FAE01452F5527469560E070E0420DF7
:104C7000531D641D751DC3010E947C25282F8823A8
:104C800009F086C0DE01B170860101701070011557
:104C9000110551F0F301EA0FFB1F82A98F70982DC7
:104CA0009295907F982B01C0982DA60DB71DD29696
:104CB0009C93219681E0F3018483AE01452F552713
:104CC000469560E070E0420D531D641D751DC301E3
:104CD0000E947C25282F882309F05AC0D170012B0F
:104CE00049F084E0B694A794979487948A95D1F775
:104CF000482D0BC0F301EC0FFD1F42A9407FBB27DD
:104D0000AB2D9A2D892D8F70482BC60DD71D4AAB20
:104D10003FC0452F562F672F7727420D531D641D27
:104D2000751DC3010E947C25282F882389F5F60173
:104D3000EE0FFF1FF170E60DF71D82AA892D99274E
:104D400083AB26C0E7E07695679557954795EA953A
:104D5000D1F7420D531D641D751DC3010E947C25B2
:104D6000282F8823A9F4F601EE0FFF1FEE0FFF1F77
:104D7000F170E60DF71D82AA892D992783ABC50135
:104D8000AA27BB2784AB8B2D9927AA27BB2785ABE6
:104D900081E0F301848301C022E0822FDF91CF9173
:104DA0001F910F91FF90EF90DF90CF90BF90AF9049
:104DB0009F908F907F906F905F904F903F902F903B
:104DC00008957F928F929F92AF92BF92CF92DF927F
:104DD000EF92FF920F931F93CF93DF934C017A01D1
:104DE0008B01423051056105710508F4BBC0F40127
:104DF000868D978DA0A1B1A1481759076A077B0737
:104E000008F0B0C0A2A0B3A0C4A0D5A08081823019
:104E100009F44DC0833009F468C0813009F0A7C09F
:104E2000EA01D695C795CE0DDF1DAE01452F55275A
:104E3000469560E070E04A0D5B1D6C1D7D1DC40150
:104E40000E947C25882309F092C0FE01F170E80DD4
:104E5000F91D72A82196AE01452F5527469560E0B1
:104E600070E04A0D5B1D6C1D7D1DC4010E947C25F8
:104E7000882309F07CC0672D70E0D170C80DD91D62
:104E80009AA980E0682B792BC70181709070892BDB
:104E900039F094E0769567959A95E1F79B0122C0E9
:104EA0009B0140E050E03F704070507064C0452F5F
:104EB000562F672F77274A0D5B1D6C1D7D1DC40182
:104EC0000E947C25882309F052C0F701EE0FFF1FD6
:104ED000F170E80DF91D93A980E022A930E0822B42
:104EE000932B9C0140E050E046C0B7E07695679573
:104EF00057954795BA95D1F74A0D5B1D6C1D7D1DE1
:104F0000C4010E947C25882391F5F701EE0FFF1F55
:104F1000EE0FFF1FF170E80DF91D85A990E0A0E0EC
:104F2000B0E0582F44273327222784A990E0A0E03F
:104F3000B0E0DC0199278827282B392B4A2B5B2BE3
:104F400082A990E0A0E0B0E0282B392B4A2B5B2B04
:104F500093A980E0A0E0B0E0282B392B4A2B5B2BF3
:104F60005F7009C021E030E040E050E004C02FEF66
:104F70003FEF4FEF5FEFB901CA01DF91CF911F9172
:104F80000F91FF90EF90DF90CF90BF90AF909F90E8
:104F90008F907F900895AF92BF92CF92DF92EF9261
:104FA000FF920F931F93CF93DF936C015B01DC01A2
:104FB00014966D937C93159716964D915D916D9116
:104FC0007C911997413051056105710509F4CEC0F6
:104FD000ED91FC91868D978DA0A1B1A1481759073D
:104FE0006A077B0708F0C2C04115510561057105CC
:104FF00081F58081833049F446A157A160A571A550
:10500000411551056105710521F5F60112861386DA
:10501000148615860190F081E02D80859185A81673
:10502000B90608F0A3C0C501A4E096958795AA9596
:10503000E1F7A0E0B0E026A137A140A551A5820F7D
:10504000931FA41FB51FF60186879787A08BB18B8E
:105050007AC08281082F10E0F4E0000F111FFA954A
:10506000E1F724C0CE010E94E126AB01BC014F3F15
:10507000FFEF5F07FFEF6F07FFEF7F0711F481E09E
:1050800076C0423051056105710508F46FC0D60144
:10509000ED91FC91868D978DA0A1B1A1481759077C
:1050A0006A077B0708F062C0A01AB10AF601C08146
:1050B000D181A016B106B0F6D6011A964D935D9334
:1050C0006D937C931D97EEEFEE2EEFEFFE2EEFEF3C
:1050D0000E2FEFEF1E2FE40EF51E061F171F8E8DED
:1050E0009F8DA8A1B9A10297A109B109E816F906F7
:1050F0000A071B0728F020E030E040E050E012C033
:105100002A8130E040E050E0C801B7010E94095C0C
:105110009B01AC018AA59BA5ACA5BDA5280F391F95
:105120004A1F5B1FC50164E0969587956A95E1F774
:10513000A0E0B0E0280F391F4A1F5B1FF601268749
:105140003787408B518BD6018D919C91C296BFE0E1
:10515000AB22BB2455E0AA0CBB1C5A95E1F78A0D83
:105160009B1DF601828B938B80E001C082E0DF9172
:10517000CF911F910F91FF90EF90DF90CF90BF9054
:10518000AF9008952F923F924F925F926F927F92CD
:105190008F929F92AF92BF92CF92DF92EF92FF9247
:1051A0000F931F93DF93CF9300D00F92CDB7DEB74D
:1051B0001C012A013B01DC015E968D919D910D90B1
:1051C000BC91A02D89839A83AB83BC834115510583
:1051D0006105710581F4F10182849384A484B5840E
:1051E00081149104A104B10411F188169906AA064C
:1051F000BB06E8F421C0C1010E94E1269B01AC017D
:10520000623071058105910528F421E030E040E02D
:1052100050E093C089819A81AB81BC8128173907FE
:105220004A075B0708F489C05301420105C011E039
:10523000812E912CA12CB12C750164010894C11C04
:10524000D11CE11CF11C89819A81AB81BC81C816FB
:10525000D906EA06FB0660F092E089169104A104E3
:10526000B10408F461C0B2E0CB2ED12CE12CF12CBA
:10527000C101B701A6010E94E1269B01AC016115A5
:10528000710581059105A9F06F3FAFEF7A07AFEF88
:105290008A07AFEF9A0709F450C0613071058105A4
:1052A000910509F44AC0C814D904EA04FB0431F694
:1052B0003BC0BC2CAD2C9E2C8F2CC101A601B7018C
:1052C0000FEF1FEF2FEF3FE00E94F525882389F5B0
:1052D000411451046104710449F0C101B301A201F8
:1052E000860197010E94F525882319F5F101B28600
:1052F000A3869486858686859785A089B1898F3F08
:10530000FFEF9F07FFEFAF07FFEFBF0751F00197D8
:10531000A109B109F10186879787A08BB18B81E044
:105320008583A701960109C020E030E040E050E00D
:1053300004C02FEF3FEF4FEF5FEFB901CA01249692
:10534000CDBFDEBFCF91DF911F910F91FF90EF9006
:10535000DF90CF90BF90AF909F908F907F906F9095
:105360005F904F903F902F9008959F92AF92BF9281
:10537000CF92DF92EF92FF920F931F93CF93DF9321
:10538000EC017A018B01423051056105710508F489
:1053900058C08E8D9F8DA8A1B9A1481759076A07DB
:1053A0007B0708F441C04DC0CE01B801A7010E949F
:1053B000E1265B016C01611571058105910509F418
:1053C00042C081E0A816B104C104D104D1F12FEF8D
:1053D000A2162FEFB2062FEFC2062FEFD20611F45E
:1053E00081E032C0CE01B801A70100E010E020E06A
:1053F00030E00E94F525882339F58E859F85A889A0
:10540000B9898F3F2FEF92072FEFA2072FEFB20737
:1054100041F00196A11DB11D8E879F87A88BB98B86
:105420009D828601750102C0992493948E8D9F8D73
:10543000A8A1B9A1E816F9060A071B0708F4B4CF1A
:1054400002C082E001C080E0DF91CF911F910F91F7
:10545000FF90EF90DF90CF90BF90AF909F90089516
:10546000CF93DF93EC016C817D810E94CB27982F35
:10547000882399F44E855F85688979898881998127
:105480000E947C25982F882341F4EA89FB8985EEC8
:105490008083E881F98181E08483892FDF91CF9136
:1054A00008954F925F926F927F928F929F92AF92E8
:1054B000BF92CF92DF92EF92FF920F931F93CF9301
:1054C000DF93EC01D62E6C807D800894611C711CEA
:1054D0006114710409F449C18E859F85A889B98931
:1054E0000097A105B10509F440C11FE0412E512CE0
:1054F000462057204114510409F027C10196A11DEF
:10550000B11D8E879F87A88BB98B4A855B856C857B
:105510007D85E881F981411551056105710539F4F1
:10552000808591856816790608F40FC11EC18281B5
:1055300090E001979301A4E036952795AA95E1F7AD
:1055400082239323892B09F000C1CF010E94E12619
:105550007B018C01623071058105910508F407C15A
:105560008FEFE8168FEFF8068FEF08078FEF180719
:1055700009F4FFC0E881F981868D978DA0A1B1A1C2
:10558000E816F9060A071B0708F4A6C0DD2009F48F
:10559000ECC04A855B856C857D85CF010E94C22861
:1055A0007B018C01611571058105910511F487E07E
:1055B000E1C091E0E916F1040105110509F4D7C035
:1055C000AFEFEA16AFEFFA06AFEF0A07AFEF1A0731
:1055D00009F4CFC08881998140E050E060E070E03C
:1055E0000E947C25882309F0C4C0E881F981F296E5
:1055F00080E092E001C011920197BFEF8F3F9B07BF
:10560000D1F7888099808EEFA82E8FEFB82E8FEF7C
:10561000C82E8FEFD82EAE0CBF1CC01ED11EF401B9
:10562000868D978DA0A1B1A10297A109B109A816F5
:10563000B906CA06DB0628F020E030E040E050E082
:1056400015C0D40112962C9130E040E050E0C60124
:10565000B5010E94095C9B01AC01F40182A593A5F0
:10566000A4A5B5A5280F391F4A1F5B1FD4019E961C
:105670002D933D934D935C93D197DD24CC24C3941B
:105680001AC0C4828881998140E050E060E070E0F7
:105690000E947C25882309F06CC0E881F98186A5E9
:1056A00097A5A0A9B1A90196A11DB11D86A797A78D
:1056B000A0ABB1ABD394E881F9818281D81608F30D
:1056C00086A597A5A0A9B1A98D199109A109B1092C
:1056D00086A797A7A0ABB1ABEA86FB860C871D8790
:1056E000C880D9808EEF9FEFAFEFBFEFE80EF91EB5
:1056F0000A1F1B1FF601868D978DA0A1B1A10297ED
:10570000A109B109E816F9060A071B0728F020E0ED
:1057100030E040E050E015C0D60112962C9130E008
:1057200040E050E0C801B7010E94095C9B01AC0158
:10573000F60182A593A5A4A5B5A5280F391F4A1F78
:105740005B1F2E873F87488B598B6C827D828881B7
:105750009981C29605E0440C551C0A95E1F7840D29
:10576000951D8A8B9B8B80E005C084E003C082E09E
:1057700001C081E0DF91CF911F910F91FF90EF90D9
:10578000DF90CF90BF90AF909F908F907F906F9061
:105790005F904F9008956F927F928F929F92AF92F9
:1057A000BF92CF92DF92EF92FF920F931F93CF930E
:1057B000DF93EC017B0103C00894E11CF11CF701AD
:1057C00080818032C9F38F3211F08C3541F4089416
:1057D000E11CF11C1E821F82188619860AC0E8810E
:1057E000F98186899789A08DB18D8E839F83A88743
:1057F000B987F7018081803240F4CE0160E070E02B
:105800000E94CB271A8A1B8A09C190E2792E85E073
:10581000682E0C891D89F8018BE090E001C071921F
:1058200001972FEF8F3F9207D1F7F70180818E32DA
:1058300041F060E070E0CC24DD24A8E0B0E030E08E
:1058400021C0D80180E090E0F701E80FF91FE08166
:105850000196EE3231F48330910509F4DAC0ED930C
:10586000F3CFEF3229F0EC3539F0E13208F0D1C056
:10587000E13210F424E201C020E2E80EF91EF80142
:105880002387DBC0F701EC0DFD1D20810894C11CAE
:10589000D11C213208F440C02F3209F4D8C02C3575
:1058A00009F4D5C02E3219F06A177B076CF01897EF
:1058B00009F0AFC02E3209F0ACC0330F330F68E0EF
:1058C00070E0ABE0B0E0DECF27FF05C0E22FF0E0F4
:1058D000ED54F04E2081422F50E0E8E2F0E201C0AA
:1058E00031968081882329F090E084179507C1F7CD
:1058F00090C0822F81548A3110F4326006C0822F0A
:1059000081568A3110F431602052F801E60FF71FFA
:1059100020836F5F7F4FB6CF44E0672B09F479C0D7
:10592000F8018081853E09F46082189711F4330FE5
:10593000330F232F30E0C90183709070019709F471
:1059400040612C7030702430310509F44860EC0C53
:10595000FD1CF801438771C04E855F856889798990
:10596000888199810E947C25482F882319F5EA892E
:10597000FB898081882311F444E01CC0838583FD6A
:1059800014C0DF018C899D899C01F9012BE030E076
:10599000215030408FEF2F3F380761F09C9180817C
:1059A000981719F411963196F3CFCE0160E00E945A
:1059B000512A48C0EC89FD8993859470442331F0C5
:1059C000842F443041F5992341F128C0992319F5DA
:1059D000EA89FB89838584FF20C0958888242489EF
:1059E00030E02829392940E050E0A9013327222757
:1059F000B38CAA24828D90E08A299B29A0E0B0E094
:105A0000282B392B4A2B5B2B2E833F8348875987C2
:105A100000CF86E003C0842F01C085E0DF91CF91E5
:105A20001F910F91FF90EF90DF90CF90BF90AF90BC
:105A30009F908F907F906F900895CE0160E070E00E
:105A40000E94CB27482F882309F486CFB3CF40E0AC
:105A500064CFCF93DF93EC0160E070E00E94CB272E
:105A6000482F8823E9F54E855F8568897989888183
:105A700099810E947C25482F882391F5EA89FB892A
:105A8000E081E53E89F1EE2379F1CE0161E00E94EB
:105A9000512AE6CF6A897B89FB0180E290E001C050
:105AA000119201972FEF8F3F9207D1F78C899D8933
:105AB0009C01D901FB012BE030E002C08D91819364
:105AC000215030408FEF2F3F3807C1F7EC89FD8917
:105AD00083858871FB018487E881F98181E0848373
:105AE000842FDF91CF9108954E855F8568897989EC
:105AF000888199810E947C25482F882359F2F0CF14
:105B0000CF93DF93EC0194E018C0888199810E94C3
:105B10007C25982F8823E1F4EA89FB8980818823FA
:105B2000F9F0853E19F0838583FF16C0CE0160E051
:105B30000E94512A982F882359F44E855F856889E1
:105B400079894115510561057105F9F6992321F00F
:105B50001E861F86188A198A892FDF91CF91089592
:105B600094E0F6CF0F93CF93DF93EC019A01AB0152
:105B7000BC016E5C7F4F898101E00E941C4188233B
:105B800011F063E06DC0CF5CDD4F988180E02A9119
:105B9000C053D24030E0822B932B85559A4A11F0A6
:105BA00062E05EC0C559DF4F288130E040E050E040
:105BB000522F4427332722278A9190E0A0E0B0E0BB
:105BC000DC0199278827282B392B4A2B5B2B22971E
:105BD000899190E0A0E0B0E0282B392B4A2B5B2B79
:105BE0009881C956D04080E0A0E0B0E0282B392B46
:105BF0004A2B5B2B5070265431444445504011F4DD
:105C000060E02EC060E0C957DF4F288130E040E0FF
:105C100050E0522F4427332722278A9190E0A0E0BA
:105C2000B0E0DC0199278827282B392B4A2B5B2BE6
:105C30002297899190E0A0E0B0E0282B392B4A2BE5
:105C40005B2B988180E0A0E0B0E0282B392B4A2B19
:105C50005B2B5070265431444445504009F061E0BC
:105C6000862FDF91CF910F9108950F93CF93DF93FC
:105C7000EC0140E050E060E070E00E947C25882369
:105C800009F07EC08881833009F072C08D8188233D
:105C900009F46EC01EA61FA618AA19AABE016E5C42
:105CA0007F4FFB0180E092E001C0119201972FEF3E
:105CB0008F3F9207D1F7C05DDD4F85E589938AEA72
:105CC0008883C153D24082E58AAB8BAB21E62CABF3
:105CD00091E49DABCA5EDD4F82E7899389939993E6
:105CE0002883C951D2408E85C65EDD4F8883CA5154
:105CF000D2408F85C55EDD4F8883CB51D2408E85E3
:105D00009F85A889B9899D0144275527C45EDD4F29
:105D1000288321968B2F9927AA27BB278883CD51CB
:105D2000D2408A85C25EDD4F8883CE51D2408B85BA
:105D3000C15EDD4F8883CF51D2408A859B85AC857B
:105D4000BD859D0144275527C05EDD4F28832196E0
:105D50008B2F9927AA27BB278883C152D2402A8933
:105D60003B894C895D89898101E00E945B431D82EA
:105D7000898160E040E050E00E946F41811181E044
:105D8000DF91CF910F910895FC01009789F08081F8
:105D9000882371F0868197818617970749F481815E
:105DA0000E94054080FD02C080E0089583E00895D0
:105DB00089E00895CF92DF92EF92FF920F931F93A5
:105DC000CF93DF93EC016A817B81888199810E9466
:105DD000C42E182F882309F06EC06C8167FF02C0A3
:105DE00012E069C061FD02C017E065C02E813F81ED
:105DF000488559858A859B85AC85BD8528173907D7
:105E00004A075B0708F057C02A873B874C875D87A6
:105E100060626C83888199812115310541055105A6
:105E200061F44E855F85688979890E94B529182FAC
:105E30001E861F86188A198A39C04A895B896C892F
:105E40007D890E94E1266B017C018FEFC8168FEFE0
:105E5000D8068FEFE8068FEFF806B9F181E0C81693
:105E6000D104E104F10411F412E022C0E881F981C7
:105E7000868D978DA0A1B1A1C816D906EA06FB06AA
:105E8000D0F44A895B896C897D89CF010FEF1FEFC0
:105E90002FEF3FE00E94F525182F882349F48881D1
:105EA0009981B701A6010E94B529182F112319F075
:105EB0008C8180688C83812FDF91CF911F910F910E
:105EC000FF90EF90DF90CF90089511E0F1CFEF9227
:105ED000FF920F931F93DF93CF93CDB7DEB72C972D
:105EE000CDBFDEBF8C017B01FC01628173818081AB
:105EF00091810E94C42E882359F5CE010196F801A4
:105F0000848B958BE114F10431F4C80160E070E0FA
:105F10000E94CB271DC0C8010E94802D843031F41F
:105F2000F80116861786108A118A02C0882381F428
:105F3000C801B7010E94D324C80160E00E94512A21
:105F4000843031F4F80116861786108A118A80E0B1
:105F50002C96CDBFDEBFCF91DF911F910F91FF90A7
:105F6000EF9008952F923F924F925F926F927F929F
:105F70008F929F92AF92BF92CF92DF92EF92FF9259
:105F80000F931F93DF93CF93CDB7DEB72597CDBF88
:105F9000DEBF8C839D833A014B01DC0112966D912B
:105FA0007C9113978D919C910E94C42E8B838823A2
:105FB00009F0B7C1EC81FD81848187FD92C0AC817D
:105FC000BD811A96AD90BD90CD90DC901D97A61422
:105FD000B704C804D90410F481FF02C0640153015E
:105FE000EC81FD812681378140855185168217829B
:105FF000108611868FEF8583A114B104C104D104EA
:1060000009F45BC10190F081E02DE983FA8382817C
:10601000682E77248824992409E0660C771C881C54
:10602000991C0A95D1F72115310541055105C1F19A
:1060300019012A0108942108310841085108C601B4
:10604000B5016150704080409040A40193010E94CE
:106050004F5C79018A01C201B101A40193010E9440
:106060004F5CE216F30604071507D0F0882799273E
:10607000DC0186199709A809B90982219321A42175
:10608000B521EC81FD8186839783A087B187A81A0B
:10609000B90ACA0ADB0A42895389648975893AC0F8
:1060A000AC81BD811E964D915D916D917C91519712
:1060B000411551056105710529F589819A8140E0F5
:1060C00050E060E070E00E94C228AB01BC014130AA
:1060D00051056105710541F4EC81FD818481806881
:1060E0008483F2E0FB831DC14F3F8FEF58078FEF92
:1060F00068078FEF7807B1F1EC81FD8146875787FC
:10610000608B718BAC81BD8152964D935D936D9385
:106110007C935597411551056105710509F059C0EA
:10612000CCC0EC81FD8184812081318181FF0DC053
:10613000C9010E94C228AB01BC014115510561058E
:10614000710541F4640153014AC0C9010E94E1266E
:10615000AB01BC014F3FFFEF5F07FFEF6F07FFEFA2
:106160007F0751F4AC81BD8114968C91149780689F
:1061700014968C93B1E096C04230510561057105CB
:1061800008F4AACFAC81BD81ED91FC91868D978DED
:10619000A0A1B1A1481759076A077B0708F09CCF57
:1061A000AC81BD8152964D935D936D937C935597D1
:1061B000FD0186819781A085B185860D971DA81D5B
:1061C000B91D86839783A087B187A618B708C8082A
:1061D000D9086A147B048C049D0408F4A2CFEC81D6
:1061E000FD8186819781A085B1858A0D9B1DAC1D9F
:1061F000BD1D86839783A087B187D601C50119E0AD
:10620000B695A795979587951A95D1F7E82E85832A
:106210008FEF91E0A0E0B0E0A822B922CA22DB22F1
:10622000A114B104C104D10409F447C08080918055
:10623000EEEFAE2EEFEFBE2EEFEFCE2EEFEFDE2E17
:10624000A40EB51EC61ED71EF401868D978DA0A183
:10625000B1A10297A109B109A816B906CA06DB06C1
:10626000C0F4228130E040E050E0C601B5010E9458
:10627000095C9B01AC01F40182A593A5A4A5B5A579
:10628000280F391F4A1F5B1F211531054105510594
:1062900059F4AC81BD8114968C9114978068149642
:1062A0008C93B2E0BB833DC02E0D311D411D511DAD
:1062B000E394EC81FD81E58204C020E030E040E021
:1062C00050E0EC81FD8186819781A085B185917038
:1062D000A070B0700097A105B10569F08689978913
:1062E000A08DB18D281739074A075B0721F0268B4F
:1062F000378B408F518FEC81FD812681378140851E
:10630000518582859385A485B58582179307A40757
:10631000B50738F4228733874487558784818062A4
:1063200084838B812596CDBFDEBFCF91DF911F91F6
:106330000F91FF90EF90DF90CF90BF90AF909F9024
:106340008F907F906F905F904F903F902F90089527
:106350000F931F93CF93DF93EC016A817B81888138
:1063600099810E94C42E982F882309F05CC08C81EB
:1063700085FF59C04A8D5B8D6C8D7D8D888199819B
:106380000E947C25982F882309F04DC00E8D1F8D0B
:10639000F8018385806283878A85848F8B85858FCA
:1063A0008A859B85AC85BD85CD01AA27BB27868FB5
:1063B0008A859B85AC85BD858B2F9927AA27BB270E
:1063C000878F8E85828F8F85838F8E859F85A88905
:1063D000B989CD01AA27BB27848B8E859F85A88983
:1063E000B989CD01AA27BB27892F9927858B0E94C0
:1063F000B918F801668B272F3327278B9C01442778
:106400005527208F692F772788279927618F8C81BF
:106410008F7D8C83E881F98181E0848388819981F3
:106420000E94352E982F892FDF91CF911F910F91C8
:106430000895CF93DF93EC010E94A831882311F4D3
:1064400018821982DF91CF9108952F923F924F9237
:106450005F926F927F928F929F92AF92BF92CF92F4
:10646000DF92EF92FF920F931F93CF93DF93EC0194
:10647000162F072F4A011901F901108211826A8132
:106480007B81888199810E94C42E782E882309F00F
:10649000A1C18C8187FD60C081FD03C0F7E07F2E24
:1064A00099C12A853B854C855D85C401A0E0B0E09B
:1064B000820F931FA41FB51F82179307A407B50768
:1064C00010F488249924812F902F9C0129016AC1FE
:1064D0002E813F8148855985DA01C9019170A070EC
:1064E000B0700097A105B10509F00CC1E881F981F0
:1064F0009D818281981708F440C02115310541051E
:106500005105A9F46E857F85888999896115710582
:1065100081059105C9F4CF0140E050E060E070E0F2
:106520000E94C2286E877F87888B998B07C04A8913
:106530005B896C897D89CF010E94C2286115710534
:106540008105910509F432C161307105810591051C
:1065500031F48C8180688C83E2E07E2E3BC16F3FFA
:10656000FFEF7F07FFEF8F07FFEF9F0709F4D8C00A
:106570006A8B7B8B8C8B9D8B1D82E881F98126A594
:1065800037A540A951A98E899F89A88DB98D281753
:1065900039074A075B0751F4CF0140E050E060E063
:1065A00070E00E947C25882309F0BAC00881198117
:1065B0002A893B894C895D892250304040405040B7
:1065C000F801868D978DA0A1B1A10297A109B1090B
:1065D000281739074A075B0708F0BBCF6280662D92
:1065E00070E080E090E00E94095C9B01AC01F80142
:1065F00082A593A5A4A5B5A5280F391F4A1F5B1F27
:10660000211531054105510509F4A3CF8D815901AB
:106610006A01A80EB11CC11CD11C7401EF2CFF240F
:10662000E694E114F10409F44AC0282F30E0C701D0
:10663000820F931F662D70E06817790718F47B01AD
:10664000E21AF30AF8018181B201A60195010E2D2B
:106650000E945B43882309F063C0E881F98126A585
:1066600037A540A951A92A193B094C095D09C70161
:10667000A0E0B0E0281739074A075B07C0F4DF0144
:10668000D29669E0220F331F441F551F6A95D1F738
:10669000F201E20FF31F9F0120503E4F02C0819193
:1066A0008D93E217F307D9F7E881F98114828D8180
:1066B0008E0D8D83B701762F6627770F59C02E81F7
:1066C0003F81488559858A859B85AC85BD8528177E
:1066D00039074A075B0778F0C80140E050E060E006
:1066E00070E00E947C258823D9F4E881F981A6A670
:1066F000B7A6C0AAD1AAAE8ABF8AC88ED98E8D810C
:106700008F5F8D83CE80DF80E884F9844E895F8936
:10671000688D798D888199810E947C25882331F04C
:106720008C8180688C837724739454C0C6019170E7
:1067300020E032E0281B390BB4012815390508F494
:10674000B9019B018E819F819170C296E881F98188
:10675000E80FF91FD20102C08D9181932150304082
:106760008FEF2F3F3807C1F7E881F98121E02483BB
:10677000460E571ECB01A0E0B0E02E813F81488538
:106780005985280F391F4A1F5B1F2E833F83488777
:106790005987F10180819181860F971F80839183B2
:1067A000861A970A8114910409F092CE2E813F81B6
:1067B000488559858A859B85AC85BD858217930759
:1067C000A407B50720F42A873B874C875D878C8117
:1067D00080628C83872DDF91CF911F910F91FF9065
:1067E000EF90DF90CF90BF90AF909F908F907F9071
:1067F0006F905F904F903F902F9008952F923F920F
:106800004F925F926F927F928F929F92AF92BF92C0
:10681000CF92DF92EF92FF920F931F93CF93DF936C
:10682000EC01162F072F4A011901F901108211827C
:106830006A817B81888199810E94C42E582E882389
:1068400009F03FC18C8187FD4CC080FD03C037E05B
:10685000532E37C12A853B854C855D858E819F816E
:10686000A885B985281B390B4A0B5B0BC401A0E036
:10687000B0E0281739074A075B0708F44901812F60
:10688000902F9C01390119C12E813F81488559857E
:10689000DA01C9019170A070B0700097A105B1052F
:1068A00009F0BFC0E881F9819D818281981750F17C
:1068B000211531054105510529F46E857F858889AB
:1068C000998907C04A895B896C897D89CF010E94BB
:1068D000E126623071058105910530F48C81806874
:1068E0008C8322E0522EEDC06F3FFFEF7F07FFEF5A
:1068F0008F07FFEF9F0709F4A2C06A8B7B8B8C8BFD
:106900009D8B1D82088119812A893B894C895D896B
:106910002250304040405040F801868D978DA0A114
:10692000B1A10297A109B109281739074A075B07E6
:10693000A8F64280642D70E080E090E00E94095C3F
:106940009B01AC01F80182A593A5A4A5B5A5280FCC
:10695000391F4A1F5B1F211531054105510509F4F7
:10696000BDCF8D8169017A01C80ED11CE11CF11CDB
:106970005401AB2CBB24A694A114B10409F44BC060
:10698000282F30E0C501820F931F642D70E0681737
:10699000790718F45B01A21AB30AF8018181B301E7
:1069A000A70196010A2D0E941C41882309F047C0C7
:1069B000E881F9818481882331F126A537A540A992
:1069C00051A92C193D094E095F09C501A0E0B0E0AD
:1069D000281739074A075B07B0F4B9E0220F331FC5
:1069E000441F551FBA95D1F7C301820F931FDF01D2
:1069F000D296FC019C0120503E4F02C08D918193A4
:106A0000E217F307D9F78D818A0D8D83B501762FB3
:106A10006627770F38C0CE8ADF8AE88EF98E8F5FBF
:106A20008D83CE80DF80E884F9844E895F89688D0C
:106A3000798D888199810E947C25882331F08C8111
:106A400080688C83552453943CC0C601917020E02B
:106A500032E0281B390BB4012815390508F4B901B7
:106A60009B018E819F819170C296E881F981E80F28
:106A7000F91FD30102C081918D93215030408FEFD7
:106A80002F3F3807C1F7660E771ECB01A0E0B0E0BC
:106A90002E813F8148855985280F391F4A1F5B1F6A
:106AA0002E833F8348875987F10180819181860F2A
:106AB000971F80839183861A970A8114910409F0A5
:106AC000E3CE852DDF91CF911F910F91FF90EF9035
:106AD000DF90CF90BF90AF909F908F907F906F90FE
:106AE0005F904F903F902F9008956F927F928F927A
:106AF0009F92AF92BF92CF92DF92EF92FF920F934D
:106B00001F93CF93DF93DC01142FED91FC9111972C
:106B10008081282F30E0205330402A30310538F46E
:106B200081818A3321F43296ED93FC9304C08091E5
:106B3000BA20282F30E0232B11F08BE085C2C091C2
:106B4000B620D091B720FB01C083D183209711F4E8
:106B50008CE07AC28881882359F089810E9405409F
:106B600080FD06C0112309F46CC282FD68C269C2AF
:106B70001882198280E00E94C94380FF02C083E02E
:106B800063C2112311F082FD5AC2CE0140E050E0F1
:106B900060E070E00E94B22D813021F0AA24BB2475
:106BA00065012FC0FE01E051FE4F8481882309F466
:106BB0004AC2838590E0A0E0B0E0D82ECC24BB246C
:106BC000AA24828590E0A0E0B0E0DC019927882724
:106BD000A82AB92ACA2ADB2A808590E0A0E0B0E082
:106BE000A82AB92ACA2ADB2A918580E0A0E0B0E071
:106BF000A82AB92ACA2ADB2ACE01B601A5010E9419
:106C0000B22D833011F481E01FC2882309F01BC22A
:106C10009EAD80E02DAD30E0822B932B80509240D2
:106C200009F011C2C75BDF4F988180E02A91C854F8
:106C3000D04030E0822B932B7C0100E010E0E11487
:106C4000F1040105110541F5C75ADF4F888190E035
:106C5000A0E0B0E0182F0027FF24EE248A9190E0F6
:106C6000A0E0B0E0DC0199278827E82AF92A0A2B5E
:106C70001B2B2297899190E0A0E0B0E0E82AF92A46
:106C80000A2B1B2B9881C755D04080E0A0E0B0E0D4
:106C9000E82AF92A0A2B1B2BEA8EFB8E0C8F1D8FFC
:106CA000CE5BDF4F2881C254D0402B8330E040E0E0
:106CB00050E0C801B7010E94095C3B014C01CF5B69
:106CC000DF4F988180E02A91C054D04030E0822B81
:106CD000932BA0E0B0E08A0D9B1DAC1DBD1D8AA3C7
:106CE0009BA3ACA3BDA38FAD8A83CC5BDF4F988100
:106CF00080E02A91C354D040422F50E0482B592BBA
:106D000048875987CA5BDF4F988180E02A91C55434
:106D1000D04030E0822B932B7C0100E010E0E114A6
:106D2000F1040105110541F5CB5ADF4F888190E050
:106D3000A0E0B0E0182F0027FF24EE248A9190E015
:106D4000A0E0B0E0DC0199278827E82AF92A0A2B7D
:106D50001B2B2297899190E0A0E0B0E0E82AF92A65
:106D60000A2B1B2B9881C355D04080E0A0E0B0E0F7
:106D7000E82AF92A0A2B1B2BCF5BDF4F988180E092
:106D80002A91C054D04030E0822B932BA0E0B0E099
:106D9000E81AF90A0A0B1B0BE618F7080809190983
:106DA000B4E056954795BA95E1F7CA01A0E0B0E086
:106DB000E81AF90A0A0B1B0B2A8130E040E050E088
:106DC000C801B7010E944F5C2E5F3F4F4F4F5F4F8E
:106DD0002E8F3F8F48A359A3273F8FE0380780E0CD
:106DE000480780E0580710F411E007C0275F3F4FC5
:106DF0004040504008F037C112E08AA19BA1ACA1ED
:106E0000BDA1860D971DA81DB91D8EA39FA3A8A780
:106E1000B9A788859985A4E096958795AA95E1F705
:106E2000A0E0B0E02AA13BA14CA15DA1820F931F7D
:106E3000A41FB51F860D971DA81DB91D8AA79BA766
:106E4000ACA7BDA78FEF9FEFAFEFBFEF8E879F87F8
:106E5000A88BB98B1C82133009F0DCC01D82CD5980
:106E6000DF4F388120E08A91C256D04090E0282B35
:106E7000392B40E050E02A0D3B1D4C1D5D1D2A8B37
:106E80003B8B4C8B5D8BBE016E5C7F4F898101E03B
:106E90000E941C41882309F0BDC0CF5CDD4F988162
:106EA00080E02A91C053D24030E0822B932B85554D
:106EB0009A4A09F0AFC02DA930E040E050E0522FCF
:106EC0004427332722278CA990E0A0E0B0E0DC0122
:106ED00099278827282B392B4A2B5B2B8AA990E0EE
:106EE000A0E0B0E0282B392B4A2B5B2B9BA980E03C
:106EF000A0E0B0E0282B392B4A2B5B2B22553245E2
:106F00004146514409F086C0C75EDD4F288130E01C
:106F100040E050E0522F4427332722278A9190E007
:106F2000A0E0B0E0DC0199278827282B392B4A2BD9
:106F30005B2B2297899190E0A0E0B0E0282B392BC1
:106F40004A2B5B2B9881C751D24080E0A0E0B0E093
:106F5000282B392B4A2B5B2B225732474144514671
:106F600009F058C0CF5DDD4F288130E040E050E0AF
:106F7000522F4427332722278A9190E0A0E0B0E0E7
:106F8000DC0199278827282B392B4A2B5B2B22974A
:106F9000899190E0A0E0B0E0282B392B4A2B5B2BA5
:106FA0009881CF51D24080E0A0E0B0E0282B392B6F
:106FB0004A2B5B2B2A873B874C875D87C35EDD4F5F
:106FC000288130E040E050E0522F44273327222729
:106FD0008A9190E0A0E0B0E0DC0199278827282B77
:106FE000392B4A2B5B2B2297899190E0A0E0B0E0EF
:106FF000282B392B4A2B5B2B9881CB51D24080E038
:10700000A0E0B0E0282B392B4A2B5B2B2E873F8743
:10701000488B598B18831EA61FA618AA19AA1E8A68
:107020001F8A188E198E8091B8209091B9200196F0
:107030008093B8209093B9208E839F8302C08AE00A
:1070400003C080E001C08DE0DF91CF911F910F91CF
:10705000FF90EF90DF90CF90BF90AF909F908F9078
:107060007F906F900895CF59DF4F288130E040E046
:1070700050E0522F4427332722278A9190E0A0E046
:10708000B0E0DC0199278827282B392B4A2B5B2B72
:107090002297899190E0A0E0B0E0282B392B4A2B71
:1070A0005B2B9881CF55D04080E0A0E0B0E0282B4A
:1070B000392B4A2B5B2B2EA33FA348A759A713E0DC
:1070C000A8CECF92DF92EF92FF920F931F93DF93A0
:1070D000CF93CDB7DEB7CF54D040CDBFDEBF8E014A
:1070E000025B1F4FD8018D939C936B01CE010196DB
:1070F0008EAB9FAB82E2E82EF12CEC0EFD1EC80198
:10710000B70141E00E947535882309F0FBC08AA1D0
:107110009BA188AF99AFF80160817181C7010E947E
:10712000CB2B882309F0EEC0EEA9FFA9838585FF4C
:1071300002C086E0E7C08CA99DA9009711F484E005
:10714000E1C0DC01FE013D9604C01A968C911A97AD
:1071500081931196EE15FF05C1F7DE01D896F70170
:107160009D0102C081918D93E217F307D9F78E013B
:10717000085C1F4FC801B6010E94CB2B882311F475
:1071800088E0C0C0843009F0BDC0C8010E94292D2C
:10719000882309F0B7C0FE01E65BFF4F40815181B3
:1071A000DA01FE013F9604C081911C968C931C97D6
:1071B0001196EE15FF05C1F78D858062DA011B96E9
:1071C0008C931B97EAA1FBA181E084831B968C9191
:1071D0001B9784FF8BC0C8ACD9AC5A962C915A9798
:1071E00030E054968C91549790E0282B392B55968B
:1071F0009C91559780E0282B392B5B969C9180E0E1
:10720000282B392B790100E010E08EEF9FEFAFEFD4
:10721000BFEFE80EF91E0A1F1B1FF601868D978D22
:10722000A0A1B1A10297A109B109E816F9060A07C0
:107230001B0708F066C0228130E040E050E0C80142
:10724000B7010E94095CAB01BC01F60182A593A5C0
:10725000A4A5B5A5480F591F6A1F7B1F41155105ED
:107260006105710509F44DC0C6010E947C25A8ADD9
:10727000B9AD882309F046C0BD016E5A7F4FFB01AE
:1072800081818E3299F58C918330B1F4FE01FE96A6
:10729000208131814281538196968D919D910D90EF
:1072A000BC91A02D281739074A075B0729F420E075
:1072B00030E040E050E006C0FE01FE9620813181C2
:1072C00042815381DB015A962C935A97832F992739
:1072D0005B968C93CA01AA27BB27FB01848B892F5D
:1072E0009927858BE8ADF9AD81E08483CE01829644
:1072F0000E94302A882331F48AA19BA10E94352E56
:1073000001C082E0C15BDF4FCDBFDEBFCF91DF9117
:107310001F910F91FF90EF90DF90CF900895EF9223
:10732000FF920F931F93DF93CF93CDB7DEB7A49750
:10733000CDBFDEBF8BA39CA38B019DE0E92EF12C7A
:10734000EC0EFD1ECE018396B70141E00E9475351B
:10735000882369F5CE01019689A39AA36BA17CA12C
:10736000C7010E94CB2B882311F5E9A1FAA18385DF
:1073700085FD1CC0EF8DF8A13097C1F0D80116969D
:107380008C911697868B17968C911797878B1496EE
:107390008C911497808F15968C91818FED85FE8549
:1073A00081E08483CF010E94352E01C086E0A4963F
:1073B000CDBFDEBFCF91DF911F910F91FF90EF9076
:1073C0000895EF92FF920F931F93DF93CF93CDB762
:1073D000DEB7A497CDBFDEBF8BA39CA3E62EF42E11
:1073E0008E01035F1F4FCE018396B80141E00E94DA
:1073F0007535882331F5CE01019689A39AA36BA137
:107400007CA1C8010E94CB2B8823D9F4E9A1FAA161
:10741000838585FD15C0EF8DF8A1309789F09F2DEC
:107420009772892F8095238582239E21892B8387BC
:10743000ED85FE8581E08483CF010E94352E01C059
:1074400086E0A496CDBFDEBFCF91DF911F910F9153
:10745000FF90EF9008952F923F924F925F926F921C
:107460007F928F929F92AF92BF92CF92DF92EF92D4
:10747000FF920F931F93DF93CF93CDB7DEB7AC97F7
:10748000CDBFDEBF8BA39CA37DE0E72EF12CEC0EDD
:10749000FD1ECE018396B70141E00E947535182F7D
:1074A000882309F053C1CE01019689A39AA36BA149
:1074B0007CA1C7010E94CB2B182F882351F0843068
:1074C00009F044C1E9A1FAA1838585FF04C016E053
:1074D0003DC118E03BC18D859E8540E050E060E0F5
:1074E00070E00E94C2284B015C01611571058105A5
:1074F000910511F417E02AC16130710581059105EC
:1075000011F412E023C16F3F3FEF73073FEF830792
:107510003FEF930709F431C18D859E8540E050E02F
:1075200060E070E00E947C25182F882309F00EC1CE
:107530000D851E856EEFC62E6FEFD62E6FEFE62EF1
:107540006FEFF62EC80CD91CEA1CFB1CF801868DC7
:10755000978DA0A1B1A10297A109B109C816D906BA
:10756000EA06FB0620F044245524320114C0F80139
:10757000228130E040E050E0C701B6010E94095C82
:107580002B013C01F80182A593A5A4A5B5A5480E41
:10759000591E6A1E7B1E52E3252E312C200E311EF1
:1075A000F10180E092E001C0119201972FEF8F3F2F
:1075B0009207D1F7F1018BE090E020E201C0219326
:1075C00001973FEF8F3F9307D1F78EE2F80182AB2F
:1075D00080E185AF0E94B9186CA7085B1F4FF801C6
:1075E0006193272F33272BA721939C0144275527ED
:1075F0002AA72193692F77278827992769A761935D
:1076000088A681928F01892D99278FA38083C50138
:10761000AA27BB278EA307501040F80181938F0142
:10762000892F99278DA3808307541040F10120E210
:1076300030E003C0808180A33196215030408FEF2D
:107640002F3F3807B9F70D5A1F4F8EE2F80180839C
:10765000035510402B893C894D895E89ED85FE8557
:107660008081833069F486A197A1A0A5B1A52817D0
:1076700039074A075B0721F420E030E040E050E0A2
:1076800004591F4FF80121938F01832F992780837D
:10769000CA01AA27BB2707501040F8018193892F00
:1076A000992780837301620101E01FC0C6A6D7A697
:1076B000E0AAF1AA0483CF0140E050E060E070E06E
:1076C0000E947C25182F882309F040C0F10180E03A
:1076D00092E001C0119201972FEF8F3F9207D1F7EF
:1076E0000894C11CD11CE11CF11CED85FE859C2D6C
:1076F000941982819817D0F2CE010D960E94292DFF
:10770000182F882339F08D859E85B501A4010E942C
:10771000B5291CC0EF8DF8A180E183873CA5368B8D
:107720008BA5878B2AA5208F39A5318F88A5828FBD
:107730002FA1238F3EA1348B8DA1858BED85FE85F6
:1077400081E08483CF010E94352E182F812FAC96C3
:10775000CDBFDEBFCF91DF911F910F91FF90EF90D2
:10776000DF90CF90BF90AF909F908F907F906F9061
:107770005F904F903F902F90089511E0E7CFCF9208
:10778000DF92EF92FF920F931F93DF93CF93CDB7CA
:10779000DEB7EA97CDBFDEBF89AF9AAF0DE0C02E4E
:1077A000D12CCC0EDD1ECE01C996B60141E00E945F
:1077B0007535882309F077C0CE01019689A39AA375
:1077C00069AD7AADC6010E94CB2B882309F06BC04E
:1077D000E9A1FAA1838585FD63C0EF8DF8A13097FB
:1077E00009F45EC08385482F80FD5CC0958980E0E8
:1077F000248930E0822B932BA0E0B0E08C01FF24A1
:10780000EE24938D80E0228D30E0822B932BA0E03C
:10781000B0E0E82AF92A0A2B1B2B44FF29C082E09A
:10782000E816F1040105110510F482E03CC0DE0108
:107830009396F6019D0102C081918D93E217F307A3
:10784000D9F7E9A6FAA60BA71CA7E3E2CE2ED12C06
:10785000CC0EDD1EC60162E070E00E94CB278823BB
:1078600011F5C6010E94802D8823E1F08430D9F4FF
:10787000CE010D960E94302A8823A9F4E114F10468
:107880000105110541F08D859E85B801A7010E9473
:10789000B529882341F48D859E850E94352E03C02D
:1078A00086E001C087E0EA96CDBFDEBFCF91DF91D1
:1078B0001F910F91FF90EF90DF90CF9008952F923E
:1078C0003F924F925F926F927F928F929F92AF9270
:1078D000BF92CF92DF92EF92FF920F931F93DF93AD
:1078E000CF93CDB7DEB72997CDBFDEBF89839A830B
:1078F0006C837D832A01CE010196BA0140E00E948B
:107900007535882309F0EBC0D201ED91FC912685F5
:10791000378540895189E68CF78C00A111A1D801E7
:10792000C7010297A109B10982179307A407B507F8
:1079300038F0EC81FD812083318342835383CEC0B4
:1079400030803B82232D2130E1F5AA24BB24650140
:1079500092E0E92EF12C012D112DD2018D919C91F7
:10796000B801A7010E94E1266F3FBFEF7B07BFEF81
:107970008B07BFEF9B0711F481E0B1C06130710547
:107980008105910511F482E0AAC061157105810598
:10799000910529F40894A11CB11CC11CD11C0894A8
:1079A000E11CF11C011D111DD201ED91FC91868D90
:1079B000978DA0A1B1A1E816F9060A071B0768F286
:1079C0007BC062A073A084A095A0AA24BB246501FB
:1079D00060E070E0E0E0F0E061157105A9F4F2010B
:1079E00080819181B401A3010E947C25882309F044
:1079F00076C00894611C711C811C911CD201ED9110
:107A0000FC91F29660E072E0B181B887208129870D
:107A10003B81323099F4BF831E82822F90E0AE8189
:107A2000BF818A2B9B2B892B29F40894A11CB11CA4
:107A3000C11CD11C32966250704033C0238130E0AB
:107A400040E050E0522F442733272227828190E0E4
:107A5000A0E0B0E0DC0199278827282B392B4A2B9E
:107A60005B2B3984832D90E0A0E0B0E0282B392BEC
:107A70004A2B5B2B38842224C101A0E0B0E0282BE4
:107A8000392B4A2B5B2B5F702115310541055105C0
:107A900029F40894A11CB11CC11CD11C349664505B
:107AA00070400894E108F10801091109E114F1049A
:107AB0000105110509F090CFD201ED91FC91A68648
:107AC000B786C08AD18ABB81B33011F481E0858347
:107AD000EC81FD81A082B182C282D38280E02996AE
:107AE000CDBFDEBFCF91DF911F910F91FF90EF903F
:107AF000DF90CF90BF90AF909F908F907F906F90CE
:107B00005F904F903F902F900895CF92DF92EF9229
:107B1000FF921F93DF93CF93CDB7DEB7A497CDBF6E
:107B2000DEBF8BA39CA36B012DE0E22EF12CEC0EAB
:107B3000FD1ECE018396B70140E00E947535182FD7
:107B40008823B1F4CE01019689A39AA36BA17CA1ED
:107B5000C7010E94CB2B182F882351F48F8D98A139
:107B6000892B11F416E004C0C701B6010E94D3248A
:107B7000812FA496CDBFDEBFCF91DF911F91FF90E3
:107B8000EF90DF90CF9008950F931F93DF93CF93E3
:107B9000CDB7DEB72E97CDBFDEBF8C016D877E8758
:107BA000CE010D96B80140E00E947535882309F09A
:107BB00046C0CE010196D80154968D939C9355975B
:107BC0006D857E85C8010E94CB2B8823A9F5D8013D
:107BD0005296ED91FC9153973097F9F0838584FF8D
:107BE0002DC0358920E0848990E0282B392B40E096
:107BF00050E0A90133272227938D80E0628D70E049
:107C0000862B972BA0E0B0E0282B392B4A2B5B2B3F
:107C1000F8012683378340875187D801ED91FC9185
:107C200011978681978112968D939C931397C80123
:107C300060E070E00E94CB27843009F485E02E9646
:107C4000CDBFDEBFCF91DF911F910F910895EF92CD
:107C5000FF921F93DF93CF93CDB7DEB7A497CDBF2D
:107C6000DEBF8BA39CA3EDE0EE2EF12CEC0EFD1EEF
:107C7000CE018396B70140E00E947535182F882306
:107C800009F044C0CE01019689A39AA36BA17CA1FF
:107C9000C7010E94CB2B182F8823A9F5AF8DB8A15F
:107CA000109739F4ED85FE85168A178A108E118E8D
:107CB0002DC01B968C911B9784FF27C0ED85FE85F8
:107CC00055963C91559720E054968C91549790E0AE
:107CD000282B392B40E050E0A901332722275B965F
:107CE0009C915B9780E05A966C9170E0862B972B65
:107CF000A0E0B0E0282B392B4A2B5B2B268B378B4F
:107D0000408F518F03C0843009F415E0812FA49671
:107D1000CDBFDEBFCF91DF911F91FF90EF9008950F
:107D20005F926F927F928F929F92AF92BF92CF920B
:107D3000DF92EF92FF920F931F93DF93CF93CDB714
:107D4000DEB7A497CDBFDEBF3C016BA37CA3DC01F3
:107D50001D921C926FE1562E54228E01035F1F4F1D
:107D60004E71CE018396B8010E947535882311F0BB
:107D7000282F37C1CE01019689A39AA36BA17CA1BC
:107D8000C8010E94CB2B282F452D50E0CA018C71D1
:107D90009070892B09F488C0222379F0243009F0EF
:107DA00020C1C8010E94292D282F882309F019C15C
:107DB000B8E05B2ACF8CD8A05BC052FE02C028E09E
:107DC00010C1CF8CD8A0C114D10409F407C1F601A9
:107DD0008385817109F002C153FE4AC0958980E014
:107DE000248930E0822B932BA0E0B0E08C01FF24AB
:107DF000EE24938D80E0228D30E0822B932BA0E047
:107E0000B0E0E82AF92A0A2B1B2B148A158A128E55
:107E1000138E148E158E168E178EED85FE8581E0DD
:107E2000848386A497A4A0A8B1A8E114F104010555
:107E30001105A1F0CF01B801A7010E94B529282F93
:107E4000882309F0CEC0ED85FE850894E108F1088D
:107E500001091109E286F386048715878D859E85C1
:107E6000B501A4010E947C25282F882309F0B9C000
:107E700053FE2CC0D6011B961C920E94B918F60125
:107E80006687272F332727879C0144275527208B78
:107E9000692F772788279927618BED85FE8581E0FB
:107EA0008483F0E25F2A12C0222309F09AC0CF8CAB
:107EB000D8A0C114D10409F493C0D6011B968C91AB
:107EC00084FD8EC051FE02C080FD88C0ED85FE8518
:107ED00026A537A540A951A9D3015A962D933D93C4
:107EE0004D935C935D978F8D98A15E968D939C9337
:107EF0005F9714965C92D60155963C91559720E079
:107F000054968C91549790E0282B392B40E050E008
:107F1000A901332722275B969C915B9780E05A96B4
:107F20006C9170E0862B972BA0E0B0E0282B392BCA
:107F30004A2B5B2BD3011E962D933D934D935C935F
:107F40005197D6015F962C915F9730E040E050E06A
:107F5000522F4427332722275E968C9190E0A0E091
:107F6000B0E0DC0199278827282B392B4A2B5B2B83
:107F7000D6015C968C9190E0A0E0B0E0282B392BE4
:107F80004A2B5B2BD6015D969C9180E0A0E0B0E08F
:107F9000282B392B4A2B5B2BD3011A962D933D931B
:107FA0004D935C931D9716961D921D921D921C92E7
:107FB00019978FEF15968C93159756961D921D92D3
:107FC0001D921C925997ED93FC931197868197818E
:107FD00012968D939C93139720E003C027E001C075
:107FE00024E0822FA496CDBFDEBFCF91DF911F91F9
:107FF0000F91FF90EF90DF90CF90BF90AF909F9048
:108000008F907F906F905F900895882311F081E0AA
:1080100008958091B32008958091BB20882319F0A2
:1080200081508093BB208091BC20882319F081501F
:108030008093BC200895AF92CF92EF920F93E0E827
:10804000F6E080E18583818380E4828380E896E0A6
:1080500060E440E020E008E1EE240E9490138EEB03
:1080600090E260EC7AE040E856E020E000E0CC24CA
:1080700033E0A32E0E944E120F91EF90CF90AF905D
:10808000089582E38093BC208EEB90E26FEF0E9414
:1080900032138EEB90E26FEF0E943213982F8F3FD6
:1080A00021F08091BC208823A1F7892F08950F9398
:1080B0001F93CF93DF938C01EB0184E18093BB206E
:1080C0008EEB90E26FEF0E9432138F3F29F4809184
:1080D000BB208823A9F71FC08E3FE9F49FEFE091F2
:1080E000BE20F091BF209383828187FFFDCF8381E3
:1080F000F8018083219719F00F5F1F4FF0CF8EEBAF
:1081000090E26FEF0E9432138EEB90E26FEF0E94CD
:10811000321381E001C080E0DF91CF911F910F9178
:10812000089580E1E0E8F6E085838EEB90E26FEF62
:108130000E943213089580E1E0E8F6E086830E9411
:1081400041408F3F11F481E008950E94914080E00A
:1081500008950E949B400E9491408091B3208160CD
:108160008093B3200895DF92EF92FF920F931F93B5
:10817000D82E7A018B0187FF0CC087E740E050E0E2
:1081800060E070E00E94B340823008F04FC08FE79B
:10819000D8220E9491400E949B40882311F48FEFC7
:1081A00045C08EEB90E26D2D0E943213212F3327B4
:1081B000442755278EEB90E2622F0E9432139801DC
:1081C000442755278EEB90E2622F0E9432135527E9
:1081D000412F302F2F2D8EEB90E2622F0E94321311
:1081E0008EEB90E26E2D0E94321380E4D81611F4CB
:1081F00065E906C088E4D81611F467E801C061E0BB
:108200008EEB90E20E9432138CE4D81629F48EEBA8
:1082100090E26FEF0E9432131AE08EEB90E26FEF64
:108220000E94321387FF02C01150B9F71F910F91BE
:10823000FF90EF90DF9008950F93CF93DF93EB01C2
:10824000882309F046C0002309F443C08091B3207D
:1082500080FF02C003E03EC08091BD2083FD07C0C7
:1082600079E0220F331F441F551F7A95D1F7013053
:1082700081F481E5BA01A9010E94B340882319F570
:10828000CE0160E072E00E9457408823E1F000E0F8
:108290001AC082E5BA01A9010E94B340882399F46B
:1082A000CE0160E072E00E945740882329F001501F
:1082B00019F0C050DE4FF4CF8CE440E050E060E0B5
:1082C00070E00E94B3400E949140002319F001E049
:1082D00001C004E0802FDF91CF910F910895EF92BC
:1082E000FF920F931F93DF93CF93CDB7DEB76097C5
:1082F000CDBFDEBF7A01882309F098C16430A9F4AC
:10830000FA018081813049F0813020F0823009F01B
:108310008DC106C00E94A94006C00E941B4003C038
:1083200081E0FA01818300E082C18091B32080FF67
:1083300002C003E07CC16A3009F41FC16B3050F405
:108340006130F1F06130A0F0623009F47AC063303E
:1083500069F47DC06C3009F417C16C3008F412C1A7
:108360006D3009F41FC16E3009F445C104E05BC1F2
:108370000E949B40882309F453C10E94914052C13E
:1083800089E440E050E060E070E00E94B340882360
:1083900009F046C1CE01019660E170E00E945740AD
:1083A000882309F43DC189818295869586958370DD
:1083B0007A854985813089F4872F90E00196342FA2
:1083C00020E0820F931FA0E0B0E00AE0880F991F21
:1083D000AA1FBB1F0A95D1F7CAC04295469546957C
:1083E0004370288530E0220F331F220F331F240FE4
:1083F000311D2F5F3F4F8F8190E083709070982FD9
:108400008827990F990F280F391F40E050E08E817F
:108410008F706B85661F6627661F860F8E5F737071
:10842000770F870F90E0099704C0220F331F441F76
:10843000551F8A95D2F7F7012083318342835383F6
:10844000F1C080E092E0FA0180839183EBC08091DB
:10845000BD2082FF34C08DEC40E050E060E070E071
:108460000E94B340882309F0DBC08EEB90E26FEFEF
:108470000E943213CE01019660E170E00E945740E5
:10848000882309F4CDC000E38EEB90E26FEF0E94E9
:1084900032130150C9F72B8522952F7080E190E0AF
:1084A000A0E0B0E004C0880F991FAA1FBB1F2A9547
:1084B000D2F7F70180839183A283B383B4C089E4A8
:1084C00040E050E060E070E00E94B340882309F093
:1084D000A7C0CE01019660E170E00E94574088235A
:1084E00009F49EC08091BD204B859C8581FF1CC0F6
:1084F000991F9927991F892F90E00196242F30E02A
:108500002F733070220F331F820F931F2E852295F9
:1085100026952695237030E02150304002C0880F08
:10852000991F2A95E2F721C0292F30E0237030707F
:10853000F3E0220F331FFA95E1F792959695977025
:10854000290F311D2F5F3F4F842F90E08C77907063
:1085500095958795959587950196AC01249FC001C7
:10856000259F900D349F900D1124A0E0B0E0F701FD
:1085700080839183A283B38355C08091BD20FA018B
:10858000808350C089E401C08AE440E050E060E0AC
:1085900070E00E94B340882309F042C0C70160E147
:1085A00070E03AC08AE740E050E060E070E00E948E
:1085B000B3408823A9F58EEB90E26FEF0E9432134F
:1085C000F70181938F018EEB90E26FEF0E943213DF
:1085D000F70181838EEB90E26FEF0E943213F80176
:1085E00081838EEB90E26FEF0E9432130F5F1F4F7B
:1085F000F801818317C08DEC40E050E060E070E04E
:108600000E94B340882361F48EEB90E26FEF0E94EA
:108610003213C70160E470E00E945740882311F4D0
:1086200001E001C000E00E94914001C004E0802F01
:108630006096CDBFDEBFCF91DF911F910F91FF906C
:10864000EF9008951F93CF93DF93EC01162F0E94B4
:1086500041408F3F11F090E029C08EEB90E2612FF6
:108660000E9432131D3F09F110E08EEB90E2688109
:108670000E943213698122968EEB90E20E9432139F
:10868000115099F78EEB90E26FEF0E9432138EEB50
:1086900090E26FEF0E9432138EEB90E26FEF0E9438
:1086A000321390E08F71853009F491E0892FDF91CA
:1086B000CF911F910895CF92DF92EF92FF920F9387
:1086C000CF93DF93EB0169017A01882309F057C04A
:1086D000002309F454C08091B32080FF02C003E05E
:1086E0004FC08091B32082FF02C002E049C0809158
:1086F000BD2090E083FD07C029E0CC0CDD1CEE1C02
:10870000FF1C2A95D1F7013079F488E5B701A6015D
:108710000E94B340882369F5CE016EEF0E94224388
:10872000882339F100E025C086709070892B39F0DC
:10873000402F50E060E070E087ED0E94B34089E593
:10874000B701A6010E94B340882399F4CE016CEFD3
:108750000E942243882329F0015019F0C050DE4FB7
:10876000F5CF80E090E06DEF0E942243882309F46A
:1087700001E00E949140002319F001E001C004E0F3
:10878000802FDF91CF910F91FF90EF90DF90CF90EE
:108790000895AF92CF92DF92EF92FF920F931F93C3
:1087A000DF93CF9300D00F92CDB7DEB7882311F0BF
:1087B00081E0C3C08091B32081FDBDC00E941B40F9
:1087C0008EEB90E260EC7AE040E856E020E000E0DA
:1087D000EE24CC24E3E0AE2E0E944E120AE08EEB93
:1087E00090E26FEF0E9432130150C9F780E440E03D
:1087F00050E060E070E00E94B340813009F07EC03C
:1088000084E68093BB2088E44AEA51E060E070E0AF
:108810000E94B340813009F04AC07E010894E11CF7
:10882000F11C870135E0C32ED12CCC0EDD1E8EEB62
:1088300090E26FEF0E943213F80181938F01EC15E3
:10884000FD05A9F78B81813009F058C08C818A3AE7
:1088500009F054C08091BB20882349F089EE40E0A4
:1088600050E060E070E40E94B340882399F7809163
:10887000BB20882309F442C08AE740E050E060E072
:1088800070E00E94B3408823C9F58EEB90E26FEF51
:108890000E943213F70181937F01E017F107A9F7D6
:1088A000898186FD02C014E02AC01CE028C089EE40
:1088B00040E050E060E070E00E94B340823018F089
:1088C00001E411E002C009EE12E08091BB20882390
:1088D00049F0802F40E050E060E070E00E94B3403B
:1088E000882399F78091BB20882341F080E540E000
:1088F00052E060E070E00E94B340811110E01093FC
:10890000BD200E9491401123A1F08091B3208E7F61
:108910008093B3208EEB90E260EC7AE040E856E082
:1089200020E000E0EE24CC24C394AA240E944E123E
:1089300002C00E94A9408091B3202496CDBFDEBF23
:10894000CF91DF911F910F91FF90EF90DF90CF902B
:10895000AF900895DC01FB01108211824CE09D91E3
:10896000292F20532A3028F0892F81548630A0F4F3
:10897000275030E0042E02C0220F331F0A94E2F782
:1089800080819181820F931F80839183442311F40E
:1089900081E008954450E3CF80E00895FC0180E039
:1089A00090E130E014C0293311F421E401C02F5FBD
:1089B000681B790B68177907B0F720833F5F343065
:1089C00041F0319624E0969587952A95E1F720E3CA
:1089D000F1CF0895E091DE2BF091DF2B8193E093AE
:1089E000DE2BF093DF2B0895EF92FF920F931F93EE
:1089F000DF93CF9300D00F92CDB7DEB79C01E62E68
:108A000060FD06C08E010D5F1F4F92E0F92E05C07C
:108A10008E010F5F1F4F84E0F82ECE010196B90141
:108A20000E94CE44D8018D91E091DE2BF091DF2B96
:108A30008193E093DE2BF093DF2B8A2F801B8F1521
:108A400090F3E1FE06C08AE08193E093DE2BF09381
:108A5000DF2B2496CDBFDEBFCF91DF911F910F9109
:108A6000FF90EF900895982F8091B420882319F0FB
:108A7000892F0E94010A0895FF920F931F93F82EE9
:108A8000062F10E004C08F2D0E9433451F5F101782
:108A9000D0F31F910F91FF9008951F93182F8BE132
:108AA0000E9433458BE50E943345812F0E94334558
:108AB0008DE60E9433451F9108958BE10E94334556
:108AC0008BE50E94334582E30E9433458AE40E948D
:108AD000334508956F927F928F929F92AF92BF928B
:108AE000CF92DF92EF92FF920F931F93CF93DF937A
:108AF000FC01C42E11E0DD2400E0E62EFF2443E05B
:108B0000A42EB12CAE20BF2034E0632E712C6E2039
:108B10007F2020E1822E912C8E209F209F012F5FAD
:108B20003F4FA114B10419F48491E90120C0808160
:108B3000FCCFC016A1F46114710481F48114910476
:108B400051F0E091DE2BF091DF2B1193E093DE2BBF
:108B5000F093DF2B03C0812F0E943345D394A114DF
:108B6000B10419F4FE01849101C088812196912FEE
:108B7000182FFE018A3011F08823D9F60F5F1123D8
:108B800069F6E4FE0AC0E091DE2BF091DF2B8AE06B
:108B90008193E093DE2BF093DF2BE3FC02C00D2DDD
:108BA00003C09A3009F40150802FDF91CF911F91BB
:108BB0000F91FF90EF90DF90CF90BF90AF909F907C
:108BC0008F907F906F90089560E040E00E946A452A
:108BD00008951F93182F80E302C08F5F1456143638
:108BE000E0F70E94334580E302C08F5F1A501A30CD
:108BF000E0F70E943345812F805D0E9433451F912D
:108C000008950F931F93182F062F8BE10E94334571
:108C10008BE50E943345812F0E94E9458BE30E943A
:108C20003345802F0E94E94588E40E9433451F9117
:108C30000F9108950E945D450E94D30987E061E08D
:108C40000E9401460E94DF4A08952F923F924F9260
:108C50005F926F927F928F929F92AF92BF92CF92CC
:108C6000DF92EF92FF920F931F93DF93CF93CDB7D5
:108C7000DEB7E797CDBFDEBF8B8B9C8B6D8B7E8B7A
:108C80004F8B288F302E30E0C90180769070898B11
:108C90009A8BA4E096958795AA95E1F7888B863004
:108CA00019F4F8E0FF8301C08F83C90180719070CF
:108CB00088879987F4E095958795FA95E1F7EDEF28
:108CC000E81BEA871F86F88DF170FAA7C901847046
:108CD00090708BA79CA7988D9095991F9927991FA5
:108CE000990F9DA7F901E270F070EEA7FFA7C901E7
:108CF0008471907088AB99ABFF81EF2FF0E0EAAB05
:108D0000FBAB3197ECABFDABC901887090708EABBB
:108D10009FAB01C0312E0E945D450E94D309EB89B3
:108D2000FC89309721F0CF01FAA5FE8304C080EEC4
:108D30009BE222E02E833889363019F4E8E04E2E8B
:108D400001C048886E816C6040E00E946A45482FEF
:108D50004E5F4D83EBA5FCA5EF2B99F02885398557
:108D6000232B11F083E001C08DA5442019F033E0DE
:108D70003D8703C04D814E5F4D879D81980F9D8338
:108D80000BC0E885F985EF2B19F4F3E0FD8704C0EB
:108D90008D5F8D8323E02D871092B4204D81242F89
:108DA00030E0C901029662E070E00E943C5C709580
:108DB00061957F4F862F845F8A8391E09E8755243B
:108DC0005394222423941C8699241B86F9013297FC
:108DD000EE8FFF8FC901019788A399A3ED858E2F90
:108DE00090E0632C77249C01260D371D2AA33BA31A
:108DF000089461087108F301E80FF91FECA3FDA3C3
:108E00000894611C711C242D30E02EA33FA3FC01AB
:108E10003197E8A7F9A779C12B893C89211531053C
:108E200019F02B833C8306C080EE9BE28B839C83EE
:108E300092E09E838824E52DEF5FE98F3E85232F06
:108E400030E02A8F3B8F452D41504C8F852D83502C
:108E50008D8F2FC18394882D90E0442019F4ECA1CC
:108E6000FDA111C02E8D3F8D821793072CF4ECA12C
:108E7000FDA18E179F0751F028A139A182179307F2
:108E80003CF0EAA1FBA18E179F0711F487E301C014
:108E900080E30E944D45182D120D812F698D0E948F
:108EA0000146F1E08F16C1F42B85921610F460E0B4
:108EB00006C0692D66956F5F3B853695631B650D12
:108EC000812F0E9401468D899E896AA54F890E9443
:108ED0006A45C82E8B8774C042E0841609F46FC0BF
:108EE00083E08816F9F4E885F985EF2B09F490C240
:108EF0002BA53CA5232B09F08BC285E590E10E94B0
:108F0000E445C82EFF24092D10E0081B110904C0F8
:108F100080E20E943345F3948F2D90E080179107F3
:108F2000BCF34EC0882D90E0E8A5F9A58E179F07E9
:108F300039F42BA53CA5232B19F0442019F43FC08C
:108F4000442029F0EE8DFF8D8E179F07C1F1FD851E
:108F50008F1639F42BA53CA5232B19F0442041F0A2
:108F600002C04420F1F0E8A1F9A18E179F07C9F4CF
:108F7000692D669528853985232B41F03D8D630F3A
:108F8000812F0E9401468FE590E107C04C8D640F50
:108F9000812F0E9401468AE590E10E94E445C82E97
:108FA0000FC08D81881609F033C2E8A9F9A974971A
:108FB00009F02EC2692D6695FC8D6F0FE9CFCC2488
:108FC00000E070C0442019F080E30E944D4510E09D
:108FD000EA8CFB8CEC18F10804C080E20E94334557
:108FE0001F5F812F90E08E159F05BCF34420C9F1CF
:108FF000082D10E0035010402EA13FA1029F7001E8
:10900000039FF00C129FF00C11240D5F1F4F80EE98
:109010009BE2E80EF91EDD247EEFA72E7FEFB72E30
:10902000A00EB11E9F859D1529F46A147B0411F4CE
:1090300085E301C080E30E944D45F70181917F01E6
:109040000E943345D394D41468F302501040601644
:10905000710611F487E301C080E30E944D45042DA1
:1090600008C04A85480D80EE9BE262E00E946A4596
:10907000082FF92CFE85FF1AF01A03C0F92CFC18F2
:1090800000E010E004C080E20E9433451F5F1F151E
:10909000D0F38C2D90E001962B813C81280F391F55
:1090A0002B833C839C1408F49C2C3C85301708F4DB
:1090B0000C874D81841608F4CDCE8A81873018F450
:1090C00067E0262E01C02A80EEA5FFA5EF2B59F000
:1090D000F92DFC5FFE878091B420882321F42C8534
:1090E000920E34E0930E892D90E0049662E070E0D9
:1090F0000E943C5C709561957F4F58E2552E560E4C
:109100008091B4208F5F8093B4208091B42082300E
:1091100008F482CE80E30E944D45C52CCA940D818F
:109120000F5F192D1D5F822D6C2D0E9401468BE271
:109130000E943345B12EBC0C822D6B2D0E9401463E
:109140008BE20E943345D22CD00E8D2D6C2D0E94C7
:1091500001468AE20E9433458D2D6B2D0E94014607
:109160008AE20E943345EC2CFF24E10EF11C122D03
:109170001E5F16C0822D652D0E9401468DE20E9461
:109180003345812F652D0E9401468DE20E943345B3
:109190008D2D652D0E9401468DE20E94334553942A
:1091A000852D90E08E159F052CF3122D1F5FE02E6C
:1091B000FF24E20CF11C0FC0812F6C2D0E94014690
:1091C0008CE70E943345812F6B2D0E9401468CE76E
:1091D0000E9433451F5F812F90E08E159F0564F339
:1091E00086E061E00E940146442019F01D81135081
:1091F00003C0102F4D85141B0E94DF4A888D87FF06
:1092000003C01092E12F88C01982CE0101960E94FE
:109210009C0B482F50E04130510511F459811DC07D
:109220008091E02F8130A1F0813018F0823089F5F3
:1092300021C089818B3119F0482F50E02AC081E08C
:109240008093E02FCE0101960E949C0B482F50E0A6
:1092500099814130510519F4592F40E01AC09B35CE
:10926000A1F482E08093E02FCE0101960E949C0B36
:10927000482F50E099814130510571F3892F815475
:10928000843018F4592F40E002C0492F50E010926A
:10929000E02F4D30510589F4E989FA89EF2B49F027
:1092A000812F90E00197232D30E0281739070CF427
:1092B00046C08DE08093E12F94C0442309F03FC065
:1092C0005093E12F513449F43A9409F024CD2EA95A
:1092D0003FA9232B09F41ECD82C0523469F4339484
:1092E000131508F018CD8EA99FA9892B11F0312EE6
:1092F00078C0332433940FCD543461F4E989FA896A
:10930000EF2B09F46EC0FF85FF2309F404CDF15063
:10931000FF8701CD533411F0332463C029893A8982
:10932000232B09F45EC03F85832F90E0ECA9FDA9B3
:109330008E179F070CF0EFCC3F5F3F87ECCC29895D
:109340003A89232B09F4E7CC632D70E0812F90E05C
:109350000197681779070CF0DECC3F858F813817AD
:1093600098F5CA01C0970A9750F0CA0181549040FD
:10937000069728F0CA0181569040069728F5CA0141
:1093800081569040069710F4405250409F85292FF7
:1093900030E061507040EAA9FBA96E9FC0016F9F49
:1093A000900D7E9F900D1124F901E052F44DE80FCD
:1093B000F91F40838CA99DA9281739070CF0ABCC65
:1093C0009F859F5F9F87A7CC4830510509F0A3CCAC
:1093D000EF85EE2309F49FCCE150EF879CCC33243A
:1093E0003394832DE796CDBFDEBFCF91DF911F91E0
:1093F0000F91FF90EF90DF90CF90BF90AF909F9034
:109400008F907F906F905F904F903F902F90089536
:109410008B819C816E8140E00E946A45C82E2EA5FA
:109420003FA5232B09F0CECD29CEAF92BF92CF928C
:10943000DF92FF920F931F93DF93CF9300D00F9291
:10944000CDB7DEB78C01F62E6A01FA016081718119
:109450005E010894A11CB11CC5010E94CE44898103
:109460008093E02B8A818093E12B8B818093E22B88
:109470008C818093E32B88E690E1B8014F2D26E59F
:1094800001E00E9425468823A9F0833011F081E095
:1094900011C08091E02B89838091E12B8A83809198
:1094A000E22B8B838091E32B8C83C501B6010E9454
:1094B000AA4482E02496CDBFDEBFCF91DF911F91F9
:1094C0000F91FF90DF90CF90BF90AF900895AF9233
:1094D000BF92CF92DF92FF920F931F93DF93CF93B0
:1094E00000D000D0CDB7DEB78C01F62E6A01B3E014
:1094F000AB2EB12CAC0EBD1EFA016081C50170E02F
:109500000E94CE448D818093E02B8E818093E12B4D
:1095100088E690E1B8014F2D26E301E00E94254640
:109520008823A1F0833011F081E010C08091E02BFE
:109530008D838091E12B8E83C501BE016F5F7F4FCC
:109540000E94AA448981F601808382E02696CDBFDD
:10955000DEBFCF91DF911F910F91FF90DF90CF90F1
:10956000BF90AF900895DF93CF930F92CDB7DEB742
:109570000E945D450E94D3098CE061E20E94014691
:1095800087E490E10E94E44586E061E00E940146A4
:109590000E94DF4A0E94FC09882341F0CE01019617
:1095A0000E949C0B813031F082E005C00E94460988
:1095B0008130F1F680E00F90CF91DF91089508950A
:1095C00090E05DE24FE410C02091DE2B3091DF2B64
:1095D000981719F4F901419302C0F9015193E093EE
:1095E000DE2BF093DF2B9F5F961770F3E091DE2B5D
:1095F000F091DF2B8AE08193E093DE2BF093DF2B59
:109600000895282FE091DE2BF091DF2BCF01805EB3
:109610009B42805094402CF42193E093DE2BF093F6
:10962000DF2B08951F920F920FB60F9208B60F927C
:109630000BB60F92112418BE1BBE2F933F938F932E
:109640009F93EF93FF938091D8329091D932892BD9
:10965000F1F08091993290919A32FC01EE0FFF1F48
:10966000E652FD4C20813181E0E0F3E0208F318F24
:10967000019690708093993290939A328091D8326B
:109680009091D93201978093D8329093D932FF913B
:10969000EF919F918F913F912F910F900BBE0F9063
:1096A00008BE0F900FBE0F901F9018956F927F927B
:1096B0008F929F92AF92BF92CF92DF92EF92FF92E2
:1096C0000F931F93CF93DF93B9E1AB2EB2E3BB2E81
:1096D00000E616E0AFE06A2E77247394F2E08F2E56
:1096E000E4E09E2E78E0E72E61E0C62ED12CA7C0E4
:1096F0004091A9325091AA3288EB92E369E172E37A
:109700002AED34E30E94FE33882311F082E0A0C0EA
:109710002091DA343091DB348091A9329091AA32D1
:109720002817390711F081E093C0A0921732B09248
:109730001832FF248091A332A0911732B0911832D1
:109740008830A9F4FD01819190E080589040582F15
:109750004427E0931732F09318328091A032823080
:1097600011F53196E0931732F09318321CC0FD01C9
:109770008191482F50E0E0931732F0931832119600
:10978000DC911197C0E04C2B5D2B3196E0931732A2
:10979000F09318328091A032823029F41496A0936D
:1097A0001732B093183280919B32F80166821416FA
:1097B0001506C4F4FFE0413A5F07A4F0F801758292
:1097C000F7E241315F0774F0F8018582F2E449362F
:1097D0005F0744F0F8019582FDE5413C5F0714F016
:1097E000F801E582F8942091153230911632B601D5
:1097F00002C0660F771F8A95E2F7CA010E943C5C9F
:1098000060507048F901EE0FFF1FE652FD4C608377
:1098100071832F5F3F4F3070209315323093163293
:109820008091D8329091D93201968093D83290931A
:10983000D9327894F394F0E2FF1609F07BCF80914F
:10984000D8329091D932813E910508F451CF80E011
:10985000DF91CF911F910F91FF90EF90DF90CF900C
:10986000BF90AF909F908F907F906F90089580E011
:1098700060E070E00E945F25089580E00E94C94387
:10988000882341F480E062EE7FE20E945F2590E051
:10989000882309F491E0892F0895FF920F931F9375
:1098A00000E01AE088E0F82EF801F1862091A1325C
:1098B0003091A23240E050E060E078E488EE91E040
:1098C0000E944F5CF80126A337A380E09AE061E094
:1098D0000E94041288EB92E34CE250E060E070E0FA
:1098E0000E94B22F882349F580E093E060E041E0D8
:1098F0000E94735280E090E8E0E0F3E0808F918F67
:1099000010921532109216321092993210929A32A9
:109910001092D8321092D9320E94564B823069F0A0
:10992000E0ECF7E0F58281E08093C52080E09AE0EA
:1099300061E00E94C41181E001C080E01F910F919D
:10994000FF90089580E09AE060E00E94C411E0E09A
:10995000F3E080818E7F808388E0E0ECF7E086830F
:109960001092C5208FE0E0E6F6E0868308950F931D
:109970008CE091E16DEE70E140E024E001E00E94B6
:1099800025460E94A24C88EB92E30E94193280E0A7
:1099900060E070E00E945F250F9108958091A832E9
:1099A000813011F40E94A24C88EB92E30E9419329C
:1099B000982F882311F481E0089580E0993009F40C
:1099C00081E008950F931F93DF93CF9300D000D0D1
:1099D000CDB7DEB780EE9BE28093DE2B9093DF2B3A
:1099E0008BEA92E38093A5329093A63262E140E045
:1099F0000E946A458091A1329091A2328E010F5F40
:109A00001F4FB8014AE050E00E94C65CC80162E105
:109A100040E00E946A458091A33290E0B8014AE09C
:109A200050E00E94C65CC80162E140E00E946A45C5
:109A30008091A03290E0B8014AE050E00E94C65CFC
:109A4000C80162E140E00E946A4585EB90E160EA6E
:109A500070E140E026E001E00E9425462696CDBF59
:109A6000DEBFCF91DF911F910F910895FF920F9369
:109A70001F93DF93CF93CDB7DEB7AE97CDBFDEBFD9
:109A80008C010E94CE4C882309F4B4C088EB92E389
:109A9000B80141E00E94903E882309F0ABC08E01DE
:109AA0000D5F1F4F88EB92E3B8014CE250E09E013E
:109AB0002F5F3F4F0E94FE33882309F09BC08981AE
:109AC0009A818C9711F0FF247AC0C80168E471E193
:109AD00044E050E00E949F5C8C01CE010B9663E451
:109AE00071E144E050E00E949F5C892B11F0FF245B
:109AF00005C0FF24012B11F4FF24F394CE010F962F
:109B00006EE371E144E050E00E949F5C892B09F014
:109B1000FF24CE01879669E371E144E050E00E94A2
:109B20009F5C892B09F0FF248F89813009F0FF2485
:109B3000898D8093A032833008F0FF249C8D80E0D3
:109B40002B8D30E0822B932B8093A1329093A23205
:109B50008DA18093A332883019F0803109F0FF2461
:109B60002CA530E040E050E0542F432F322F222725
:109B70008DA590E0A0E0B0E0DC0199278827282B94
:109B8000392B4A2B5B2B8BA590E0A0E0B0E0282B73
:109B9000392B4A2B5B2B8EA590E0A0E0B0E0B82FCC
:109BA000AA2799278827282B392B4A2B5B2B209310
:109BB0009C3230939D3240939E3250939F328091DD
:109BC000A3328695869586952091A032829F802D1E
:109BD00011248093143290E025E0880F991F2A9574
:109BE000E1F78093A9329093AA3280E0FF2019F424
:109BF00081E001C082E0AE96CDBFDEBFCF91DF91A4
:109C00001F910F91FF9008952F923F924F925F9274
:109C10006F927F928F929F92AF92BF92CF92DF927C
:109C2000EF92FF920F931F93DF93CF93CDB7DEB7E1
:109C3000AD97CDBFDEBF4C011982CE014896BE0163
:109C40006F5F7F4F0E94C43D882309F0A3C08091BD
:109C5000C620882319F400E010E020C00F920F9274
:109C600085E591E1ADB7BEB711968D939C931297A0
:109C70000E941B58E091DE2BF091DF2BCF01805E1C
:109C80009B420F900F908050944034F48AE081936F
:109C9000E093DE2BF093DF2B01E010E0EE24FF24B5
:109CA000CC24DD2488E1682E712C6C0E7D1EBDE471
:109CB0002B2EB1E13B2EABE04A2E512C4C0E5D1EFB
:109CC000FCE0AF2EB12CA80CB91C01C0CC24C30100
:109CD000BE016E5F7F4F0E94672F882309F05AC034
:109CE0008B85882309F47EC08E3289F3DD2011F440
:109CF0000F5F1F4F8A8590E09C012071307084FFB8
:109D000003C0DD2021F00FC0E1E0DE1661F4EA14AB
:109D1000FB0408F067C0E814F90410F0CC24C394E5
:109D20000894E11CF11CCC2091F2232B19F480E261
:109D300090E002C084E490E000D000D0EDB7FEB720
:109D40003196ADB7BEB711962D923C921297828391
:109D50009383448255820E941B58E091DE2BF09140
:109D6000DF2BCF01805E9B422DB73EB72A5F3F4F6E
:109D70002DBF3EBF805094400CF0A8CF8AE0819365
:109D8000E093DE2BF093DF2BA1CFD394A2E0DA1681
:109D900019F09DCF00E010E0E091DE2BF091DF2B79
:109DA000CF01805E9B42805094402CF41192E0934E
:109DB000DE2BF093DF2BC801AD96CDBFDEBFCF9178
:109DC000DF911F910F91FF90EF90DF90CF90BF90A8
:109DD000AF909F908F907F906F905F904F903F904B
:109DE0002F900895C30160E070E00E94672F8823E0
:109DF00061F2D0CF7F928F929F92AF92BF92CF921B
:109E0000DF92EF92FF920F931F93CF93DF93109205
:109E1000AB321092A4321092A83285E08093A73220
:109E20008AEE94E48093C7209093C8200E943D4C12
:109E3000882351F484EF90E16DEE70E140E024E07E
:109E400001E00E9425467FC1E0E6F6E08FE08683D0
:109E5000818301E0EE24FF2440EEA42E4BE2B42ED9
:109E60003BEAC32E32E3D32E2AE0722E9924939438
:109E700096E0892EA092DE2BB092DF2BC092A53205
:109E8000D092A632C60162E140E00E946A4580910C
:109E9000A73267E00E94E04A8091A832813019F42D
:109EA00089E291E104C0882331F481E391E160E12A
:109EB00040E00E946A45E091DE2BF091DF2B719229
:109EC000E093DE2BF093DF2B82E890E167E770E10F
:109ED00040E022E00E942546082F882369F4809103
:109EE000E12F823009F422C1813009F028C10E949B
:109EF000A24C1092A83223C1813009F0CAC0A092AE
:109F0000DE2BB092DF2BC7010E94044EEC010097BC
:109F100009F40CC180E090E06DED70E140E028E1D3
:109F20000E942546182F823008F492C08091E12FBC
:109F30008D3009F08DC0A092DE2BB092DF2BC09245
:109F4000A532D092A63292E00CC0E091DE2BF091C7
:109F5000DF2B8191E093DE2BF093DF2B8A30A9F782
:109F60009F5F911790F3E091DE2BF091DF2B9191A1
:109F700001C03196E093DE2BF093DF2BE091DE2BD6
:109F8000F091DF2B80818032A1F30EC0E091A532E9
:109F9000F091A6328193E093A532F093A632119608
:109FA000A093DE2BB093DF2BA091DE2BB091DF2BA3
:109FB0008C91803211F08A3049F7E091A532F0910E
:109FC000A6321082C092A532D092A6329434E1F427
:109FD000C6010E94273E882309F0A8C0C6016AE591
:109FE00071E142E050E00E949F5C2091C620892BE5
:109FF00011F4215001C02F5F2093C620E091A532BB
:10A00000F091A632108241C0C6010E94364D8230C6
:10A0100009F48CC08130A9F488E191E16DEE70E122
:10A0200040E024E001E00E9425461092A432E09135
:10A03000A532F091A632108288EB92E30E94193289
:10A0400026C09092A4321092A8320E94E24C77C0AF
:10A050008091E12F813439F4E114F104C1F00894C6
:10A06000E108F10814C0823459F4CD30D10578F0FC
:10A070002C97EC16FD0658F40894E11CF11C07C05F
:10A08000113029F48D3009F45AC001E038CF012F86
:10A0900036CF823001F58091E12F843469F48091CC
:10A0A000A732882309F44DC081508093A732982DA0
:10A0B000981B90939B32DECE833409F042C080918E
:10A0C000A7328630F0F58F5F8093A732982D981BCA
:10A0D00090939B3236C0833021F0843009F0CACE91
:10A0E00021C08091A8328823A9F48091A4328823CA
:10A0F00051F488E191E16DEE70E140E024E001E08F
:10A100000E9425460DC00E944D4C882379F0909204
:10A11000A83206C0813021F40E94A24C1092A832CD
:10A1200003E0A8CE0E94CE4C882319F40E94B74CBD
:10A130000AC080E060E070E00E945F2504C001E09A
:10A1400099CE02E097CEDF91CF911F910F91FF90B2
:10A15000EF90DF90CF90BF90AF909F908F907F90C7
:10A1600008959091DC3489230895FF920F931F93F3
:10A17000682F60958091DC3468236093DC3400ECB8
:10A1800017E084E0F82EF801F6828DED94E30E944A
:10A190003213F801F5821F910F91FF900895FF92FD
:10A1A0000F931F936091DC34682B6093DC3400ECD8
:10A1B00017E094E0F92EF801F6828DED94E30E9409
:10A1C0003213F801F5821F910F91FF9008956F925D
:10A1D0007F928F929F92AF92CF92EF920F931F93A5
:10A1E00030EC832E37E0932E14E0F40115831183B5
:10A1F00080E1E0EAF6E0828380EA96E060E140E018
:10A2000020E008E1EE240E9490132DED622E24E35D
:10A21000722EC30160EC7BE040EA56E020E000E0F3
:10A22000CC24AA24A3940E944E121092DC34F40190
:10A230001683C30160E00E943213F40115831F915D
:10A240000F91EF90CF90AF909F908F907F906F90F5
:10A250000895E0E0F2E08181877F818380818E7FB5
:10A2600080830895EF92FF920F931F93CF93DF9314
:10A27000C4EED4E3EE24FF2487018091230280FF03
:10A28000FCCF80E292E062E30E94E55189939993CA
:10A29000AA2797FDA095BA2FE80EF91E0A1F1B1FCB
:10A2A00084E3CC3ED80749F7C801B70124E030E089
:10A2B00040E050E00E94715CC901DF91CF911F9195
:10A2C0000F91FF90EF900895EF92FF920F931F93DD
:10A2D00080E092E00E94B25100E012E0F80181813A
:10A2E000897E806181838481887F83608483828189
:10A2F0008F7C8062828380E2E82E82E0F82EF70174
:10A300008081807E8260808389E08183F801808102
:10A310008160808380E092E00E940B5280E092E0B6
:10A3200060E272E041E00E943E528093EC34F8011A
:10A3300080818E7F808388E0F7018183F8018381AB
:10A340008F73838380818160808380E092E00E94AC
:10A350000B52F8018181886081831F910F91FF90DA
:10A36000EF900895DC0182E0A030B80781F482E02C
:10A370008093CA01E0E2F0E0E4911092CA011C96D9
:10A38000EC931C978093CA01E1E2F0E00FC082E0F9
:10A390008093CA01E4E2F0E0E4911092CA011C96B5
:10A3A000EC931C978093CA01E5E2F0E0E4911092EF
:10A3B000CA011D96EC930895FC0181E083832481FA
:10A3C0003581261B3109C9010895FC0181E0838391
:10A3D00024813581772767FD7095261B370BC901CE
:10A3E0000895FC0181E0838324813581C9010895AA
:10A3F000FC0181E0838384810895FC0181E08383F3
:10A4000085810895FC0184811482A0E0B2E0119757
:10A41000F1F784830895FC01948181E08483A0E0B6
:10A42000B4E01197F1F794830895FB014423D9F028
:10A4300020E030E040E050E061E08081806880838F
:10A44000838180FFFDCF638384819581280F391F2D
:10A450004F5F5F4F4430510581F73695279536950C
:10A460002795822F0895808180688083838180FF73
:10A47000FDCF81E08383848195810895FB0144238E
:10A48000D9F040E050E020E030E061E08081806879
:10A490008083838180FFFDCF638384819581480F12
:10A4A000591F2F5F3F4F2430310581F7CA0164E007
:10A4B00070E00E943C5C0BC0808180688083838157
:10A4C00080FFFDCF81E0838384819581682F862F73
:10A4D0000895AAECB1E092E09C93E82FF0E0E491BB
:10A4E0001C928E2F0895FC0181818F798183828156
:10A4F000867E682B642B62838081827F8560808367
:10A5000008950F93FC0181818F798064818382811A
:10A51000867E682B642B6283022B048380818D608E
:10A5200080830F910895FC01442319F4608F718F8B
:10A530000895628F738F0895FC018581662319F455
:10A5400021E030E002C022E030E040E090E028234B
:10A550003923232B09F041E0842F0895FC018181E8
:10A560008C7F862B8183477043830895682B642BEF
:10A57000622B609340040895FC01362F818127707F
:10A58000887F822B8183662757FD6095762F452F24
:10A59000562F672F7727232F269526958FEF9FEF2E
:10A5A00002C0880F991F2A95E2F78423952382839E
:10A5B0009383808180788160832B80830895FC0160
:10A5C000362F81812770887F822B8183662757FDF4
:10A5D0006095762F452F562F672F7727232F2695A7
:10A5E00026958FEF9FEF02C0880F991F2A95E2F7FB
:10A5F0008423952382839383808180788260832B58
:10A60000808308956F927F928F92AF92CF92EF9254
:10A610000F931F93DF93CF93CDB7DEB7182F3B0176
:10A620005E85A889B9896A897B8930914104442370
:10A6300011F490E001C098E0222311F480E001C001
:10A6400084E0307F302B932B892BE0E4F4E081838E
:10A65000CE28CA28C08658298F85582B5187B370B9
:10A66000A483B5837F736683778380915D04887F3D
:10A67000858F9301442737FD4095542F232F342F86
:10A68000452F5527612F669566958FEF9FEF02C086
:10A69000880F991F6A95E2F782239323868F978FFD
:10A6A00080915C0480788360812B848F80915D042D
:10A6B00087FFFCCFCF91DF911F910F91EF90CF904B
:10A6C000AF908F907F906F9008952F923F924F920E
:10A6D0005F926F927F928F929F92AF92BF92CF9232
:10A6E000DF92EF92FF920F931F935B016C011901B0
:10A6F0002A0185E5F501CBBE80831BBE21E030E059
:10A7000040E050E065E50EC0DA01C9018A0D9B1DED
:10A71000AC1DBD1DFC01ABBF60831BBE220F331FF0
:10A72000441F551F221533054405550568F38AEA71
:10A73000F501CBBE80831BBEA1E0EA2EF12C012DDA
:10A74000112D11C0A80197012A0D3B1D4C1D5D1D47
:10A75000F9014BBF80811BBE853509F05BC0EE0C53
:10A76000FF1C001F111FE214F3040405150550F32C
:10A7700085E5F501CBBE80831BBE21E030E040E0E3
:10A7800050E07AEA65E539C039014A016A0C7B1C60
:10A790008C1C9D1CF3018BBE70831BBEF501CBBED0
:10A7A00080811BBE853509F033C0E1E0EE2EF12C2F
:10A7B000012D112D15C0E216F3060407150761F0EF
:10A7C000D801C7018A0D9B1DAC1DBD1DFC01ABBF8F
:10A7D00080811BBE8535E1F4EE0CFF1C001F111FAC
:10A7E000E214F3040405150530F3F3018BBE608316
:10A7F0001BBE220F331F441F551F2215330544056E
:10A80000550508F4C1CF2FEF3FEF4FEF5FEF02C0C8
:10A81000A4019301B901CA011F910F91FF90EF901C
:10A82000DF90CF90BF90AF909F908F907F906F9070
:10A830005F904F903F902F9008952F923F924F92AC
:10A840005F926F927F928F929F92AF92BF92CF92C0
:10A85000DF92EF92FF920F931F93DF93CF9300D07D
:10A860000F92CDB7DEB769837A838B839C831901FE
:10A870002A01EE24FF24870121E0A22EB12CC12C55
:10A88000D12C19C069817A818B819C816E0D7F1DCD
:10A89000801F911FA60195010E94BC550894A11C20
:10A8A000B11CC11CD11C84E090E0A0E0B0E0E80E37
:10A8B000F91E0A1F1B1FE214F3040405150510F30B
:10A8C00066247724430191E0A92EB12CC12CD12C10
:10A8D00029C0E980FA800B811C81E60CF71C081D59
:10A8E000191DC801B7010E94AC556A157B058C057E
:10A8F0009D0509F055C0A60195012095309540951C
:10A900005095C801B7010E94BC550894A11CB11C08
:10A91000C11CD11C84E090E0A0E0B0E0680E791E7C
:10A920008A1E9B1E621473048404950490F2EE2424
:10A93000FF24870181E0A82EB12CC12CD12C27C087
:10A9400069807A808B809C806E0C7F1C801E911E9B
:10A95000C401B3010E94AC55A60195012095309524
:10A9600040955095621773078407950719F0840185
:10A97000730116C00894A11CB11CC11CD11C84E039
:10A9800090E0A0E0B0E0E80EF91E0A1F1B1FE214E1
:10A99000F30404051505A0F2EE24EA94FE2C8701C9
:10A9A000B701C8012496CDBFDEBFCF91DF911F91C3
:10A9B0000F91FF90EF90DF90CF90BF90AF909F905E
:10A9C0008F907F906F905F904F903F902F90089561
:10A9D0006F927F928F929F92AF92BF92CF92DF92AF
:10A9E000EF92FF920F931F93CF93DF93962E872EB4
:10A9F000782E692E262F372F482F592FC901DA01BB
:10AA00007C018D01C0E0D0E051E0A52EB12CC12C1D
:10AA1000D12CA60195010C2E04C0220F331F441F18
:10AA2000551F0A94D2F7C801B7010E94BC5584E0B3
:10AA300090E0A0E0B0E0E80EF91E0A1F1B1F21966F
:10AA4000C032D10531F7292D382D472D562DC9019A
:10AA5000DA017C018D01C0E0D0E041E0A42EB12CF0
:10AA6000C12CD12CC801B7010E94AC559B01AC018F
:10AA7000D601C5010C2E04C0880F991FAA1FBB1F49
:10AA80000A94D2F7281739074A075B0709F04CC028
:10AA90002095309540955095C801B7010E94BC554E
:10AAA0002196C032D10549F084E090E0A0E0B0E00A
:10AAB000E80EF91E0A1F1B1FD5CF292D382D472D53
:10AAC000562DC901DA017C018D01C0E0D0E031E0F2
:10AAD000A32EB12CC12CD12CC801B7010E94AC55BA
:10AAE000A60195010C2E04C0220F331F441F551FD1
:10AAF0000A94D2F7209530954095509562177307C8
:10AB00008407950789F42196C032D10549F084E085
:10AB100090E0A0E0B0E0E80EF91E0A1F1B1FDCCF9A
:10AB2000EE24EA94FE2C8701B701C801DF91CF9192
:10AB30001F910F91FF90EF90DF90CF90BF90AF905B
:10AB40009F908F907F906F900895FB018BBF219114
:10AB500030811BBEC9010895FB018BBF219131914A
:10AB6000419150811BBEB901CA010895FB018BBF01
:10AB7000419350831BBE0895FB018BBF21933193FA
:10AB8000419350831BBE089580E1E0E6F6E08583A3
:10AB90000895CF92DF92EF92FF920F931F93CF937E
:10ABA000DF938C016B01C0E0D0E080E0E82E82E111
:10ABB000F82E1DC08DEE94E36FE30E943213F8016E
:10ABC000EC0FFD1F808300D00F92EDB7FEB73196DA
:10ABD000ADB7BEB71196ED92FC92129782831382A5
:10ABE0000E941B5821960F900F900F900F90F60126
:10ABF000CC15DD05F8F2E00FF11F1082DF91CF9147
:10AC00001F910F91FF90EF90DF90CF900895CF921A
:10AC1000DF92EF92FF920F931F93CF93DF937B010D
:10AC20008C01C0E0D0E09BE0C92E92E1D92E1DC07E
:10AC30008DEE94E3D8016C910E94321300D00F92F4
:10AC4000EDB7FEB73196ADB7BEB71196CD92DC9297
:10AC50001297D8018D918D01828313820E941B5817
:10AC600021960F900F900F900F90CE15DF0500F3F7
:10AC7000DF91CF911F910F91FF90EF90DF90CF90D8
:10AC80000895EF92FF920F931F93282F7B0180E18D
:10AC9000E0E6F6E086830DEE14E3C801622F0E9421
:10ACA0003213C8016F2D0E943213C8016E2D0E940D
:10ACB00032131F910F91FF90EF900895DF92EF9262
:10ACC000FF920F931F9300E616E030E1D32EF801B8
:10ACD000D6822DEEE22E24E3F22EC70165E00E941B
:10ACE0003213C7016FE30E943213F801D58290E05E
:10ACF0001F910F91FF90EF90DF900895CF92DF9218
:10AD0000EF92FF920F931F93C82E50E6E52E56E068
:10AD1000F52E40E1D42EF701D6820DEE14E3C801E2
:10AD200061E00E943213C8016C2D0E943213F701BA
:10AD3000D5821F910F91FF90EF90DF90CF900895F3
:10AD4000AF92CF92EF920F93E0E6F6E080E1858339
:10AD500081838DEE94E360EC79E040E656E020E0FC
:10AD600000E0EE24CC24C394AA240E944E120F913A
:10AD7000EF90CF90AF900895DF92EF92FF920F93F4
:10AD80001F93DF93CF93CDB7DEB72B97CDBFDEBF39
:10AD900082E496E18093C7209093C8208AEE91E1E7
:10ADA0000E94D9570E94A0568FEC91E10E94D9577A
:10ADB00080E40E947E560E945E5600D00F922AEADE
:10ADC00031E1EDB7FEB721833283838394830E9400
:10ADD0001B580F900F900F900F908AE991E10E94FD
:10ADE000D95781E68A8382E68B8383E68C831D8232
:10ADF00082E060E070E00E94415672E0E72EF12CA4
:10AE0000EC0EFD1EC70164E070E00E94075600E6EC
:10AE100016E060E1D62EF801D58288E78A8389E7BB
:10AE20008B838AE78C831D8282E891E10E94D95747
:10AE300083E060E070E00E944156C70164E070E08A
:10AE40000E94C955F801D5820F920F928DE591E1CC
:10AE5000EDB7FEB7818392830E941B580F900F902D
:10AE6000CE0101960E949C0B2B96CDBFDEBFCF91E9
:10AE7000DF911F910F91FF90EF90DF9008950F9356
:10AE80001F93CF93DF938C01EB0106C0F8018191F2
:10AE90008F010E94421621971C161D06BCF380E804
:10AEA0009EE30197F1F7DF91CF911F910F910895E4
:10AEB0008F929F92AF92BF92CF92DF92EF92FF92CA
:10AEC0000F931F93DF93CF93CDB7DEB76897CDBFB6
:10AED000DEBF9FEF99839AE59A83E8E1F0E0EB8388
:10AEE000FC8395E09D838E834F83588769877A879B
:10AEF0000B871C872D873E87CF86D88AE98AFA8AF6
:10AF00008B8A9C8AAD8ABE8A1F8A86E0888FCE0192
:10AF1000019668E170E00E943F576896CDBFDEBFA2
:10AF2000CF91DF911F910F91FF90EF90DF90CF9025
:10AF3000BF90AF909F908F9008950F931F93DF93D2
:10AF4000CF93CDB7DEB76097CDBFDEBF9FEF9983BC
:10AF50009AE59A83E0E1F0E0EB83FC8395E09D8342
:10AF60008E834F83588769877A870B871C872D8745
:10AF70003E871F8686E0888BCE01019660E170E0F7
:10AF80000E943F576096CDBFDEBFCF91DF911F91EA
:10AF90000F9108958A3019F48DE001D08AE0FF9373
:10AFA000EF93E091C720F091C8200995EF91FF91B0
:10AFB0000895FC018591803011F0ECDFFBCF0895FE
:10AFC000FF27E0E230E247FF0CC0419597FF09C040
:10AFD000EDE26095709580959095611D711D811DC4
:10AFE000911D27FF02C0219530E350E2AA27660F8A
:10AFF000771F881F991FAA1FA41710F0A41B639521
:10B000005A95A9F7AA3008F0A95FA05DAF93F39510
:10B01000611571058105910541F7ED3211F4EF934A
:10B02000F395F21718F43F93F395FBCF8F91B2DFAE
:10B03000FA95E1F70895DF93CF93CDB7DEB7269663
:10B04000E991F9918591803021F0853229F0A2DFD4
:10B05000F9CFCF91DF91089520E0E89455915532D2
:10B06000B1F3503311F4689455915A3348F4505366
:10B0700080F3220F022E220F220F200D250FF4CF76
:10B080000EF4219589919991533609F3533729F19B
:10B09000533559F1BC0188279927E8945C3621F48F
:10B0A0008991999168945591543639F446EF7EF020
:10B0B00077FF0DC08FEF9FEF0AC055374AE039F098
:10B0C000583540E121F0523642E009F0C2CFFF93FB
:10B0D000EF9376DFEF91FF91B5CFFF93EF93FC01F4
:10B0E00081918030B9F356DFFBCFFF93EF9361DF9F
:10B0F000F1CF0B01DC01ED91FD912227332744278D
:10B100005527E8949AE001C0319660816032E1F3FE
:10B11000A8F16D3211F46894F7CF6A3378F5603393
:10B1200068F171F498E031966081613248F16236DD
:10B1300011F492E003C0683719F490E13196608110
:10B140006132F0F0613608F060526053B8F06A3056
:10B1500018F067506A3090F0691780F481E2771B2D
:10B1600008F4790F769557954795379527958A95E1
:10B17000B9F7260F381F481F581FE0CF80E001C0E5
:10B1800081E04EF466272095309540955095261F16
:10B19000361F461F561FFE93EE93D0012D933D930D
:10B1A0004D935D93112408956F927F928F929F9299
:10B1B000AF92BF92CF92DF92EF92FF920F931F93C5
:10B1C000DF93CF93CDB7DEB72B97CDBFDEBF5C014A
:10B1D0004B017A01FC0116821782838181FD08C030
:10B1E0006FEF7FEF08C142E050E0E40EF51E04C0AF
:10B1F0003E010894611C711CF501D380F401D3FC5D
:10B200008591D3FE81914F01882309F4F1C08532E5
:10B2100059F4D3FC6591D3FE61914F01653219F069
:10B22000062F10E01BC085E290E02BC0002309F43C
:10B23000DFC081E292E1602F70E00E94945C892B74
:10B2400039F4033211F4106103C00C3661F4106854
:10B25000F401D3FC0591D3FE01914F0117FFE6CF16
:10B26000002309F4C5C08AE192E1602F70E00E94DA
:10B27000945C892B51F044E050E0E40EF51E8FE31E
:10B2800090E0B5010E941E5DB7CF033629F0033769
:10B2900079F00335F1F40BC087010E5F1F4FF70102
:10B2A00080819181B5010E941E5D7801A5CF11605A
:10B2B000F701C080D18004C090E0B5010E941E5DFE
:10B2C000F60110FD859110FF81916F018823A1F790
:10B2D0008ACF043611F0093639F517FF08C0F70197
:10B2E000208131814281538184E090E00AC0F701DE
:10B2F000808191819C01442737FD4095542F82E045
:10B3000090E0E80EF91E1F7E57FF08C0509540954B
:10B31000309521953F4F4F4F5F4F1064CA01B901DF
:10B32000A3012AE030E034C00037A9F0013730F43F
:10B330000835B1F00F3609F05BC006C0053739F0AB
:10B34000083709F055C008C028E030E00CC01F7E67
:10B350002AE030E008C01061146220E130E003C050
:10B36000146020E132E017FF08C0F70160817181AD
:10B370008281938144E050E008C0F701808191818F
:10B38000BC0180E090E042E050E0E40EF51EA30135
:10B390000E94645DD82ED618012F10E006FF05C06C
:10B3A0008DE290E0B5010E941E5D04FF15C0FE0114
:10B3B000ED0DF11D8081803379F080E390E0B501DF
:10B3C0000E941E5D02FF08C000721070C801885AFA
:10B3D0009F4FB5010E941E5DDA94F301ED0DF11D42
:10B3E000808190E0B5010E941E5DDD20A9F704CFA9
:10B3F000F50166817781CB012B96CDBFDEBFCF9162
:10B40000DF911F910F91FF90EF90DF90CF90BF9051
:10B41000AF909F908F907F906F900895FC0120FDDA
:10B4200008C023FD05C022FF02C0738362835183DD
:10B4300040830895EF92FF920F931F9344FF02C041
:10B4400033E011C046FF02C034E00DC0DB01FC0157
:10B45000AA0FBB1FEE1FFF1F1094D1F76A0F7B1FAF
:10B460008E1F9F1F31E0660F771F881F991F315075
:10B47000D1F77B018C01E20EF11C011D111DA80109
:10B480009701B701CA011F910F91FF90EF900895A6
:10B490000F931F93CF93DF938C01C8010E94DC5C54
:10B4A000EC0197FD08C00E948C5C892BB1F7CE019E
:10B4B000B8010E944A5DCE01DF91CF911F910F919B
:10B4C0000895AF92BF92CF92DF92EF92FF920F93C7
:10B4D0001F93CF93DF93EC01C62E5A01122F0E94C7
:10B4E000DC5CAC018B3219F08D3251F41068CA94D7
:10B4F00009F46DC0CE010E94DC5CAC0197FD67C011
:10B500006DEFD62ED1228D2D807301F54033F1F4ED
:10B51000CA9409F447C0CE010E94DC5CAC0197FDDF
:10B5200041C082E0D82A483711F0483559F480E408
:10B53000D82ACA94B9F1CE010E94DC5CAC019923EF
:10B540002CF430C0D6FC02C080E1D82AEE24FF24BF
:10B550008701242F2053283088F0D4FC09C02A30DA
:10B5600068F0D6FE05C02F7D822F8151863028F0ED
:10B57000CA01BE010E944A5D12C02750C801B7012E
:10B580004D2D0E941A5A7B018C0182E0D82ACA9460
:10B5900061F0CE010E94DC5CAC0197FFDACFD1FCF8
:10B5A00004C015C0EE24FF248701D7FE08C0109503
:10B5B0000095F094E094E11CF11C011D111DC501E2
:10B5C000B801A7012D2D0E940E5A81E001C080E034
:10B5D000DF91CF911F910F91FF90EF90DF90CF906F
:10B5E000BF90AF9008956F927F928F929F92AF928B
:10B5F000BF92CF92DF92EF92FF920F931F93CF9360
:10B60000DF935C016B013A01FC01168217828824EA
:10B61000DDC0812F90E00E948C5C892B21F0C50158
:10B620000E94485AD3C0153249F4F601F3FC6591E3
:10B63000F3FE61916F01653269F415E2C5010E9464
:10B64000DC5C97FDCFC0181709F4C0C0B5010E949B
:10B650004A5DCDC06A3219F0162F00E006C0F3FC37
:10B660001591F3FE11916F0101E099240FC0026062
:10B67000692D70E080E090E040E20E941A5A962E18
:10B68000F601F3FC1591F3FE11916F01212F205368
:10B690002A3068F301FD03C099249A9403C09920CD
:10B6A00009F4A5C0183621F01C3699F4F6010BC038
:10B6B000F601F3FC6591F3FE6191683619F06F01B4
:10B6C000162F07C008600460F3FC1591F3FE11917A
:10B6D0006F01112309F48BC081E392E1612F70E0C7
:10B6E0000E94945C892B09F482C0802F00FF03C064
:10B6F000EE24FF2407C0F301E080F18022E030E077
:10B70000620E731E1E3651F4F5014681578160E0CA
:10B7100070E0C701202F0E940E5A58C0133691F4D2
:10B7200081FD02C099249394C5010E94DC5C97FDC1
:10B7300059C0E114F10419F0F70181937F019A9443
:10B7400099F742C0C5010E94485A97FD4BC01F3669
:10B7500059F1103728F4143629F1193639F527C074
:10B76000133719F0153711F51DC0C5010E94DC5CB7
:10B77000EC0197FD11C00E948C5C892B29F0CE0151
:10B78000B5010E944A5D08C0E114F10419F0F70107
:10B79000C1937F019A9449F7E114F104A9F0F701EC
:10B7A000108212C0006203C0006101C00064C501C4
:10B7B000692DA701202F0E94615A882329F4F501E1
:10B7C0008381807379F413C000FF8394F501F380C3
:10B7D000F601F3FC1591F3FE11916F01112309F0AD
:10B7E00018CF05C0882019F42FEF3FEF02C0282D95
:10B7F00030E0C901DF91CF911F910F91FF90EF9041
:10B80000DF90CF90BF90AF909F908F907F906F9080
:10B810000895629FD001739FF001829FE00DF11D9A
:10B82000649FE00DF11D929FF00D839FF00D749FBA
:10B83000F00D659FF00D9927729FB00DE11DF91F66
:10B84000639FB00DE11DF91FBD01CF0111240895C3
:10B85000AA1BBB1B51E107C0AA1FBB1FA617B70736
:10B8600010F0A61BB70B881F991F5A95A9F7809552
:10B870009095BC01CD01089597FB092E07260AD0AB
:10B8800077FD04D0E5DF06D000201AF470956195AD
:10B890007F4F0895F6F7909581959F4F0895A1E207
:10B8A0001A2EAA1BBB1BFD010DC0AA1FBB1FEE1F3A
:10B8B000FF1FA217B307E407F50720F0A21BB30B85
:10B8C000E40BF50B661F771F881F991F1A9469F701
:10B8D00060957095809590959B01AC01BD01CF015D
:10B8E000089597FB092E05260ED057FD04D0D7DF0B
:10B8F0000AD0001C38F450954095309521953F4F63
:10B900004F4F5F4F0895F6F790958095709561952C
:10B910007F4F8F4F9F4F0895911134C1803219F09E
:10B9200089508550D0F70895FC010590061621F046
:10B930000020D9F7C00108953197CF010895FB0188
:10B94000DC014150504030F08D910590801919F480
:10B950000020B9F7881B990B0895DC0101C06D9395
:10B9600041505040E0F70895FC018191861721F085
:10B970008823D9F7992708953197CF010895FB01BE
:10B98000DC0101900D920020E1F70895FB019F0179
:10B99000423074F0453264F4642F77270E94285CAB
:10B9A000805D8A330CF0895D8193CB010097A1F70C
:10B9B0001082C9010C94C55DCF93DF93EC014B81DC
:10B9C00040FF1AC046FF0AC04F7B4B838E819F8188
:10B9D00001968E839F838A81282F2BC042FF13C03C
:10B9E000E881F9818081282F332727FD30952115A3
:10B9F000310529F440624B832FEF3FEF1BC0319696
:10BA0000E883F98311C0EA85FB85CE0119959C0175
:10BA100097FF0AC09B812F5F3F4F11F080E201C06A
:10BA200080E1892B8B83E8CF8E819F8101968E8365
:10BA30009F8330E0C901DF91CF9108950F931F9349
:10BA4000CF93DF938C01EB018B8181FF1BC082FFC1
:10BA50000DC02E813F818C819D812817390764F4A8
:10BA6000E881F9810193E883F98306C0E885F985C7
:10BA7000802F1995892B31F48E819F8101968E83B9
:10BA80009F8302C00FEF1FEFC801DF91CF911F917D
:10BA90000F9108959C01FB01838180FF11C086FDF9
:10BAA0000FC09FEF2F3F390759F0228380648F7DAD
:10BAB00083838681978101978683978330E002C0D4
:10BAC0002FEF3FEFC9010895FA01AA27283051F15D
:10BAD000203181F1E8946F936E7F6E5F7F4F8F4FBF
:10BAE0009F4FAF4FB1E03ED0B4E03CD0670F781F1E
:10BAF000891F9A1FA11D680F791F8A1F911DA11D03
:10BB00006A0F711D811D911DA11D20D009F468943B
:10BB10003F912AE0269F11243019305D3193DEF6E3
:10BB2000CF010895462F4770405D4193B3E00FD099
:10BB3000C9F7F6CF462F4F70405D4A3318F0495D84
:10BB400031FD4052419302D0A9F7EACFB4E0A69567
:10BB50009795879577956795BA95C9F70097610589
:10BB6000710508959B01AC010A2E069457954795DF
:10BB700037952795BA95C9F7620F731F841F951FD4
:10BB8000A01D0895992788270895DC01FC01672FDF
:10BB900071917723E1F7329704C07C916D937083A4
:0EBBA0006291AE17BF07C8F30895F894FFCF67
:10BBAE0054656D70657261747572650044656720C9
:10BBBE00460054656D7000566F6C74616765006D5C
:10BBCE005600566F6C74000120222A2B2C5B3D5DB3
:10BBDE007C7F00809A90418E418F80454545494932
:10BBEE00498E8F9092924F994F555559999A9B9C89
:10BBFE009D9E9F41494F55A5A5A6A7A8A9AAABAC46
:10BC0E0021AEAFB0B1B2B3B4B5B6B7B8B9BABBBC6A
:10BC1E00BDBEBFC0C1C2C3C4C5C6C7C8C9CACBCCCE
:10BC2E00CDCECFD0D1D2D3D4D5D6D7D8D9DADBDCBE
:10BC3E00DDDEDFE0E1E2E3E4E5E6E7E8E9EAEBECAE
:10BC4E00EDEEEFF0F1F2F3F4F5F6F7F8F9FAFBFC9E
:06BC5E00FDFEFF010100E4
:00000001FF
